:020000040800F2
:10000000080C0024AD020008913D0008EB34000804
:10001000B9020008A5030008414E000800000000D6
:100020000000000000000000000000006D4100081A
:10003000C305000800000000933D00087D43000850
:10004000C7020008C7020008C7020008C70200086C
:10005000C7020008C7020008C7020008C70200085C
:10006000C7020008C7020008C7020008C70200084C
:10007000C7020008C7020008C7020008C70200083C
:10008000C7020008C7020008C7020008C70200082C
:10009000C7020008C7020008C7020008C70200081C
:1000A000C7020008C7020008C7020008C70200080C
:1000B000C7020008C7020008C7020008C7020008FC
:1000C000C7020008C7020008C7020008C7020008EC
:1000D000C7020008FD4D0008C7020008C70200085B
:1000E000C7020008C702000800000000C70200089D
:1000F000C7020008C7020008C7020008C7020008BC
:10010000C7020008C7020008C7020008C7020008AB
:10011000C7020008C7020008C7020008C70200089B
:10012000C7020008C7020008C7020008C70200088B
:10013000C7020008C7020008C7020008C70200087B
:1001400000000000000000000000000000000000AF
:10015000C7020008C7020008C7020008C70200085B
:10016000C7020008C7020008C7020008C70200084B
:10017000C7020008C7020008C7020008C70200083B
:10018000C7020008C7020008C7020008C70200082B
:10019000C7020008C7020008C7020008C70200081B
:1001A000C7020008C7020008C7020008C70200080B
:1001B000C7020008C7020008C7020008C7020008FB
:1001C000C7020008C7020008C7020008C7020008EB
:1001D000C7020008C7020008C7020008C7020008DB
:1001E000C7020008C7020008C7020008C7020008CB
:1001F000C7020008C7020008C7020008C7020008BB
:10020000C7020008C7020008C7020008C7020008AA
:10021000C7020008C7020008C7020008C70200089A
:10022000C7020008C7020008C7020008000000005B
:10023000C7020008C702000800000000C70200084B
:10024000C7020008C7020008C7020008C70200086A
:10025000C7020008C7020008C7020008C70200085A
:10026000C7020008C7020008C7020008C70200084A
:10027000C7020008C7020008C7020008000000000B
:10028000C702000800000000C702000800000000CC
:1002900000000000C7020008DFF80CD000F070F882
:1002A00000480047E94E0008080C00240648804733
:1002B00006480047FEE7FEE7FEE7FEE7FEE7FEE74B
:1002C000FEE7FEE7FEE7FEE781430008990200082B
:1002D0002DE9F05F0546002092469B46884606467B
:1002E000814640241BE0284641464746224600F00E
:1002F00036F853465A46C01A914110D31146184653
:10030000224600F01DF82D1A67EB01084F462246E1
:100310000120002100F014F817EB00094E41201EC7
:10032000A4F10104DFDC484631462A464346BDE8D5
:10033000F09F421C10F8011B0029FBD1801A704766
:10034000202A04DB203A00FA02F100207047914095
:10035000C2F1200320FA03F3194390407047202A8A
:1003600004DB203A21FA02F00021704721FA02F35F
:10037000D040C2F120029140084319467047000066
:10038000064C074D06E0E06840F0010394E80700E2
:1003900098471034AC42F6D3FFF782FF647200082E
:1003A00084720008FEE70000F0B5BFF34F8FBFF383
:1003B0006F8F1E4900200860BFF34F8FBFF36F8F10
:1003C0001B4E316841F400313160BFF34F8FBFF3F2
:1003D0006F8F174970310860BFF34F8F081F006897
:1003E000C0F34E31114A43F6FF771032C0F3C9050E
:1003F000284607EA411343EA80741460401E441CF7
:10040000F9D1491E481CF3D1BFF34F8F306840F437
:1004100080303060BFF34F8FBFF36F8F03484C3095
:10042000016841F004010160F0BD000050EF00E000
:1004300014ED00E0F8B54EF67D7003F057F81F227A
:100440001021182033A300F027FA364C4FF47845DA
:10045000009505216088401F83B22088401F82B22A
:10046000084603F0AFF94FF6E07600966088142155
:10047000143883B22088143882B2084603F0A2F9F7
:100480001F20009060883221323883B220883238B1
:1004900082B2084603F096F94FF61F00009060887C
:1004A0006421503883B22088503882B2502003F043
:1004B00089F94FF4FA6004F0EDFC4FF6FF7003F099
:1004C00015F800F019FA4FF49674204604F0E2FC97
:1004D000002003F00BF8204604F0DCFC284603F073
:1004E00005F8204604F0D6FC304602F0FFFF204617
:1004F00004F0D0FC4FF4FC6002F0F8FF204604F05A
:10050000C9FC1F2002F0F2FF2046BDE8F84004F0CD
:10051000C1BC0000313A20D1D5C9ABCCEEB3E4B2B6
:10052000E2CAD400F40100242DE9F0438146884654
:1005300015461E4600240B4F04EB041117F811005A
:10054000A84209D107EB41014878B04204D1891C87
:100550004246484600F02AF8641CA4B2382CEBD37B
:10056000BDE8F083646700082DE9F04381468846C2
:1005700015461E4600240C4F04EB840000EB44108B
:1005800017F81010A94209D107EB40014878B04292
:1005900004D1891C4246484600F008F8641CA4B205
:1005A000092CE9D3BDE8F0833A6F000810B50023A9
:1005B00004E011F8014B00F8014B5B1C9342F8D3A7
:1005C00010BD704710B54EF67D7002F08FFF4FF6EC
:1005D0001F0404212246102023A300F075F92021D6
:1005E0002246302025A300F06FF95823E022402155
:1005F000102000F07BF81F224421302022A300F0BD
:100600004BF98023E0226821102000F06FF81F22B0
:100610006C21302020A300F03FF9A823E022902194
:10062000102000F063F81F22942130201EA300F058
:1006300033F94FF47844B421224610201EA300F071
:100640002BF9C4212246102021A300F025F94FF4F4
:10065000FA6004F01FFCFFF7EDFE00F0B9F9BDE809
:10066000104000F097BA000044657645426F782D3F
:10067000B4F3D4BDB4B4D0C200000000D2BABEA757
:10068000C6C1B2E2CAD40000313A20D1D5C9ABCC40
:10069000EEB3E4B2E2CAD400323A20CEC4D7D6CF09
:1006A000D4CABEB2E2CAD400333A20CDBCC6ACCF65
:1006B000D4CABEB2E2CAD400463A206D63756465FE
:1006C000762E74616F62616F2E636F6D00000000A3
:1006D000463A2073686F70333839393537323930DC
:1006E0002E74616F62616F2E636F6D002DE9F843A8
:1006F00080460E4614461F464FF6FF753346224687
:1007000031464046009502F06BFF3B46424631467B
:100710004046009502F064FF7D1E48F2104908F142
:1007200001002246ABB2CDF80090A9B280B202F02F
:1007300057FF44F208253B4622463946404600957D
:1007400002F04EFF601E3B4682B2CDF80090711C55
:1007500089B280B202F044FF3B4622463146204631
:10076000009502F03DFFBDE8F8830000F0B585B0CC
:1007700014461D460A4B1A88121A92B25B885B1AFD
:100780009BB2084F4FF0300C00263F88CDE9005C4B
:10079000CDE90376029400F02BFC05B0F0BD00001B
:1007A000F40100241E000024F0B585B014461D4657
:1007B0000A4B1A88121A92B25B885B1A9BB2084FD6
:1007C0004FF0400C00263F88CDE9005CCDE9037670
:1007D000029400F00DFC05B0F0BD0000F40100240F
:1007E0001E000024F0B585B014461D460A4B1A8839
:1007F000121A92B25B885B1A9BB2084F4FF00C0C36
:1008000000263F88CDE9005CCDE90376029400F034
:10081000EFFB05B0F0BD0000F40100241E00002431
:10082000F0B585B014461D460A4B1A88121A92B2CA
:100830005B885B1A9BB2084F4FF0100C00263F8874
:10084000CDE9005CCDE90376029400F0D1FB05B060
:10085000F0BD0000F40100241E000024F0B585B0B6
:1008600014461D460A4B1A88121A92B25B885B1A0C
:100870009BB2084F4FF0200C00263F88CDE9005C6A
:10088000CDE90376029400F0B3FB05B0F0BD0000A3
:10089000F40100241E0000242DE9FF4114461D46EA
:1008A000084B1A88121A92B25B885B1A9BB2002618
:1008B0001027CDE90246CDE9005703F0ADFCBDE8B5
:1008C000FF810000F40100242DE9FF4114461D467C
:1008D000084B1A88121A92B25B885B1A9BB20026E8
:1008E0001827CDE90246CDE9005703F095FCBDE895
:1008F000FF810000F401002438B54FF6FF7002F0CC
:10090000F5FD8023DC22402114204FF4784400942C
:1009100002F066FE40230094DC228021142002F0C5
:100920005FFE1F2000908023DC224021142002F073
:10093000A4FE4FF61F04512223466021782002F0C6
:10094000C1FE502223466021782002F0BBFE4F22D8
:1009500023466021782002F0B5FEBDE838404FF410
:10096000FA6004F097BA00002DE9F04105460C4604
:100970001646DFF85880012240461703394600F03A
:1009800055FD052000F0C8FB032003F02FFBC4F346
:10099000074003F02BFBC4F3072003F027FBE0B272
:1009A00003F024FB002405E0FF2003F01FFB285583
:1009B000641CA4B2B442F7D300223946404600F08A
:1009C00035FDBDE8F041052000F0A6BB000402584B
:1009D00070B54EF67D74204602F088FD1F2210216E
:1009E000182026A3FFF758FF4FF47A7004F052FA4C
:1009F000204602F07BFD00220421102023A3FFF7F4
:100A000063FF00222021302025A3FFF75DFF002295
:100A10005021182025A3FFF73FFF6021182027A3AE
:100A20004FF4FC62FFF738FF1F227021182026A325
:100A3000FFF732FF4FF4784580212A46182026A37D
:100A4000FFF72AFF1F229021102027A3FFF724FF82
:100A50001F22A02110202AA3FFF71EFF2F4BB02139
:100A600010202A46FFF718FF40F6B83004F012FABB
:100A70002046BDE8704002F039BD0000323A20CE79
:100A8000C4D7D6CFD4CABEB2E2CAD4004465764534
:100A9000426F782DB4F3D4BDB4B4D0C200000000CE
:100AA000D2BABEA7C6C1B2E2CAD40000C7B6C8EB6C
:100AB000CABDBFAAB7A2CDF800000000D6D0CEC4F0
:100AC000B2E2CAD400000000D7A8D7A2D2BABEA70B
:100AD000C5FAB7A200000000C8ABB3CCBCBCCAF5D5
:100AE000D6A7B3D600000000463A206D6375646552
:100AF000762E74616F62616F2E636F6D000000006F
:100B0000463A2073686F70333839393537323930A7
:100B10002E74616F62616F2E636F6D00207200082A
:100B200030B404460D4610461A46217820281DD0C0
:100B300009DC0C2812D0102814D018281ED1104817
:100B400001FB020106E0302814D0402816D10D48E0
:100B500001FB0201284630BCFFF706BF514301F5F7
:100B60000021F7E7084801FB0201F3E7074801FB12
:100B70000201EFE7064801FB0201EBE730BC7047DA
:100B80000012080000920800000808000026080073
:100B9000004808002DE9F04186B04EF67D784046C9
:100BA00002F0A4FC1F221021182047A3FFF738FEF3
:100BB0004FF47A7004F06EF9404602F097FC484D0D
:100BC00000242021F0220B462888CDE90384CDE9BA
:100BD000011044A021460090182000F009FA454E6B
:100BE00010272988F0223B463088CDE90171CDE9F4
:100BF000030441A000902821384600F0F9F9298823
:100C000010233088F022CDE90171CDE903043EA024
:100C100000903821184600F0EBF91F2248211020DF
:100C20003FA3FFF7DFFD1F21CDE9001841A002908F
:100C3000C8230C226021102000F03AFA29880C22E7
:100C400030881346CDE9030441A0CDE90121F0220B
:100C500000907821102000F0CBF9298810233088EB
:100C6000F022CDE90171CDE903043EA00090882176
:100C7000184600F0BDF92988182230881346CDE9BE
:100C800003043CA0CDE90121F02200909C2110201A
:100C900000F0AEF91F22B821102039A3FFF7DEFDC6
:100CA0001F22DC21102039A3FFF760FD1F22DC2169
:100CB000782037A3FFF778FD06B040F6B830BDE8DE
:100CC000F04104F0E7B80000323A2047424BD7D653
:100CD000BFE22D2DCFD4CABEB2E2CAD400000000BC
:100CE00020000024CAAED6D6D7D6BFE2B2E2CAD41C
:100CF0000000000022000024C9E8BCC6A3BAB4F377
:100D0000D4BDB5E7D7D3000046726F6D3A206D634E
:100D1000756465762E74616F62616F2E636F6D000E
:100D2000446174653A20323031392F30352F3038F4
:100D300000000000BED3D6D0CFD4CABEBAAFCAFD21
:100D40003A20323031392F30352F30380000000052
:100D5000BABAD7D631327831322D47424BD7D6BFC7
:100D6000E2A3BA00BABAD7D63136783136D7D6BF71
:100D7000E2A3BA003234783234D7D6BFE2A3BA0045
:100D80003332783332D7D6BFE2A3BA00343800000A
:100D90003634000030B4054608462C786978812C3A
:100DA0000AD3402908D3FF2906D0FF2C04D07F297D
:100DB0000DD24039CDB20CE00021002203E000F852
:100DC000012B491C89B29942F9D330BC7047413993
:100DD000CDB2813CE1B2C1EB411404EB811105EBD2
:100DE000410159430C2A0BD0102A0CD0182A0DD0DF
:100DF000202AEAD101F560111A4630BCFFF7B4BDD4
:100E0000044A1144F8E7044A1144F5E701F5ED11ED
:100E1000F2E700000014090000DD1100AFF30080CC
:100E200070B586B04FF6FF7002F060FB00206D4693
:100E300000242C54401CC0B21828FAD31122684652
:100E40000021FFF791FD10216B464FF478460846CC
:100E50003246FFF7E5FC00202C54401CC0B2182895
:100E6000FAD3082268461421FFF77EFD20216B4645
:100E700010203246FFF7D4FC00202C54401CC0B296
:100E80001828FAD3082268461E21FFF76DFD30218D
:100E90006B4610203246FFF7C3FC40F6B83003F033
:100EA000F9FF06B070BD2DE9F04FC1B082460D4686
:100EB00016461C46A946600701D0012000E000202C
:100EC00000EBD40B60080BFB00FB0C2C09D0102CA2
:100ED00007D0182C05D0202C03D0302C01D0402C6A
:100EE00033D101A95B4622463046FFF719FE4FF089
:100EF000000828E001A810F808700026380605D57B
:100F00004A9A2946504602F041FC06E04C9820B926
:100F10004B9A2946504602F039FC7806070E6D1CA4
:100F2000ADB2A5EB0900A04205D14D460AF1010A78
:100F30001FFA8AFA03E0761CB6B2082EDED308F157
:100F400001081FFA88F8D845D4D341B0BDE8F08F26
:100F50002DE9F04FA1B082460C4615461F46A1462A
:100F6000780701D0012000E0002000EBD70B0BFB3D
:100F700007FB0C2F05D0102F03D0182F01D0202FE6
:100F800033D101A95B463A462846FFF703FF4FF0ED
:100F9000000828E001A810F808600025300605D5F3
:100FA0002A9A2146504602F0F1FB06E02C9820B91F
:100FB0002B9A2146504602F0E9FB7006060E641C8F
:100FC000A4B2A4EB0900B84205D14C460AF1010ACB
:100FD0001FFA8AFA03E06D1CEDB2082DDED308F18A
:100FE000010808F0FF08D845D4D321B0BDE8F08F40
:100FF0002DE9FF4F83B004460E469346DDE9107598
:10100000A046B2464FF0000920E0B9F1000F23D00E
:101010004FF0000908EB0B00401BA04202DA7019E8
:1010200086B2444606985044401BB04211DBDDE9CD
:10103000121214982B4602902046CDE900123A462F
:101040003146FFF785FFBF1C601984B2387800284D
:10105000DBD107B0BDE8F08F802802D94FF001093D
:10106000F4E708EB0B01A1EB5501A14202DA71197B
:101070008EB2444606995144491BB142E9DB0D2822
:1010800010D0DDE9121214982B4602902046CDE9CB
:1010900000123A463146FFF706FF7F1C04EB55006D
:1010A00084B2D3E7701986B244467F1CF5E700008E
:1010B0002DE9F04786B08046894614469A46DDE918
:1010C0000E67109D2846FFF734F9610841438AB244
:1010D0001049012352450CD901A8D0C000954046C3
:1010E00004934B880A884946FFF782FF06B0BDE8A3
:1010F000F087AAEB020202EBD270400801AA40443A
:1011000080B2D0C2009504934B880A884946FFF705
:101110006FFFEBE7F4010024002206E00021491CE8
:10112000C9B26429FBD3521CD2B28242F6D37047B3
:1011300030B405460846144619462A786B78812A49
:101140000FD3402B0DD3FF2B0BD0FF2A09D00C2936
:1011500010D0102910D018290CD1214630BCFFF72F
:1011600003BA0021002203E000F8012B491CC9B298
:10117000A142F9D330BC7047214630BCFFF7D4B947
:1011800010B5002807D090F83510022905D080212D
:101190004165012010BD012010BD214A4FF4956426
:1011A00001688B18A34207D8042280F8352008680C
:1011B00020F00100086030E00B6823F00E030B60A4
:1011C00001680A44A24204D80A6822F001020A60B7
:1011D00003E00A6822F001020A60016E0A6822F444
:1011E00080720A6090F85C10012404FA01F20D4943
:1011F0000A60D0E919215160C16E31B10A6822F448
:1012000080730B60D0E91C215160002180F83410FC
:1012100080F83540016D01B18847002010BD000005
:10122000F0FFFDBF045402580248016841F001017B
:1012300001607047200400582DE9F84F00226D4CE2
:101240004FF0B04A4FF001094FF0030E4FF00F0876
:1012500009FA02F70B683B40BB4270D14D68022D82
:1012600001D0122D12D1D50800EB850CDCF82060DE
:101270005507ED0E08FA05FB26EA0B06D1F810B06B
:101280000BFA05FB4BEA060BCCF820B0D0F800C0F7
:1012900055000EFA05F62CEA060C91F804B00BF096
:1012A000030B0BFA05FB4BEA0C0BC0F800B0D1F8AE
:1012B00004C0BCF1010F08D0BCF1020F05D0BCF195
:1012C000110F02D0BCF1120F16D1D0F808C02CEAD1
:1012D000060CD1F80CB00BFA05FB4BEA0C0BC0F86E
:1012E00008B0D0F804C02CEA070C0F79C7F3001738
:1012F000974047EA0C074760C768B7438E68AE401F
:101300003E43C6604D68ED006DD53B4D2E6846F0FE
:1013100002062E602D6805F00205009522F00306F6
:1013200006F1B046D6F808C495072F0F08FA07F55E
:101330002CEA050C314DA84202D100252EE052E0E6
:101340002F4DA84201D1012528E02E4DA84201D100
:10135000022523E02C4DA84201D103251EE02B4D90
:10136000A84201D1042519E0294DA84201D1052543
:1013700014E0284DA84201D106250FE0264DA842D1
:1013800001D107250AE0254DA84201D1082505E035
:10139000234DA84201D1092500E00A25BD4045EAB8
:1013A0000C05C6F8085425689D434E68F60300D521
:1013B0001D43256065689D434E68B60300D51D43F7
:1013C0006560DAF800509D434E68F60200D51D4373
:1013D000CAF80050DAF804509D434E68B60200D5B2
:1013E0001D43CAF80450521C102AFFF431AFBDE867
:1013F000F88F000080000058F444025800000258A2
:101400000004025800080258000C0258001002584C
:101410000014025800180258001C025800200258FC
:101420000024025842694A4042617047002A01D0B4
:10143000018370474183704701488068704700000E
:1014400010000024024881680278114481607047CE
:101450001000002410B5032000F05AF80F2000F00F
:1014600007F808B1012010BD00F024F8002010BDDD
:1014700070B504460D4D4FF47A712878B1FBF0F049
:101480000B490968B1FBF0F001F04AFE08B10120F8
:1014900070BD102C07D200222146501E00F018F813
:1014A0006C60002070BD012070BD000010000024A1
:1014B000000000247047002809DB012100F01F0212
:1014C00091404009800000F1E020C0F80011704711
:1014D000F0B40D460D4B1B68C3F30223C3F10704A0
:1014E000042C00D90424191D072901D2002300E08F
:1014F000DB1E012606FA04F1491E294099409E4050
:10150000761E16403143F0BC03F09BBC0CED00E0AE
:1015100000F00701054A10684FF6FF03184040EA43
:101520000120034908431060704700000CED00E003
:101530000000FA0510B500F083FF084909684FF470
:10154000807292FAA2F201F47061B2FA82F2D14092
:10155000034A515CC8400349086010BD1844025852
:101560007C4F00080000002410B500F023FF07495D
:101570000968102292FAA2F201F07001B2FA82F226
:10158000D140034A515CC84010BD000020440258BD
:101590007C4F000830B55F490A6802F00302096811
:1015A000C1F305315B4B1B1D1B6803F01003594C45
:1015B00014342468C4F3CC0414FB03F300EE103A93
:1015C000B8EE400ADFED540A524BB7EE001A103362
:1015D000002A42D0514C012A73D0022A70D0B4FBA9
:1015E000F1F101EE901A1968B8EE612AC1F3080111
:1015F00001EE901AF8EE611A40EE201A31EE810ADF
:1016000022EE000A1968C1F34621491C00EE901A27
:10161000F8EE600A80EE201AFCEEC10AC0ED000A66
:101620001968C1F30641491C00EE901AF8EE600AF1
:1016300080EE201AFCEEC10AC0ED010A1968C1F360
:101640000661491C00EE901AF8EE600A80EE201A3E
:10165000BCEEC10A80ED020A30BD2E4C283C226847
:1016600095062F4A17D52468C4F3C104E240B2FBA3
:10167000F1F101EE901A1968B8EE612AC1F3080180
:1016800001EE901AF8EE611A40EE201A31EE810A4E
:1016900022EE000AB6E7B2FBF1F101EE901A1968EA
:1016A000B8EE612AC1F3080101EE901AF8EE611A52
:1016B00040EE201A31EE810A22EE000AA2E700E095
:1016C00013E0B4FBF1F101EE901A1968B8EE612A4B
:1016D000C1F3080101EE901AF8EE611A40EE201AEB
:1016E00031EE810A22EE000A8CE70E4AB2FBF1F1DC
:1016F00001EE901A1968B8EE612AC1F3080101EEF3
:10170000901AF8EE611A40EE201A31EE810A22EEAC
:10171000000A77E7284402580000003900093D001C
:101720000090D00340787D0130B55F490A6802F02F
:1017300003020968C1F305515B4B1B1D1B6803F4D1
:101740008073594C1C342468C4F3CC0414FB03F399
:1017500000EE103AB8EE400ADFED540A524BB7EEF5
:10176000001A1833002A42D0514C012A73D0022AA1
:1017700070D0B4FBF1F101EE901A1968B8EE612A4D
:10178000C1F3080101EE901AF8EE611A40EE201A3A
:1017900031EE810A22EE000A1968C1F34621491C84
:1017A00000EE901AF8EE600A80EE201AFCEEC10AF4
:1017B000C0ED000A1968C1F30641491C00EE901AF9
:1017C000F8EE600A80EE201AFCEEC10AC0ED010AB4
:1017D0001968C1F30661491C00EE901AF8EE600A20
:1017E00080EE201ABCEEC10A80ED020A30BD2E4CFC
:1017F000283C226895062F4A17D52468C4F3C104F3
:10180000E240B2FBF1F101EE901A1968B8EE612ADC
:10181000C1F3080101EE901AF8EE611A40EE201AA9
:1018200031EE810A22EE000AB6E7B2FBF1F101EED9
:10183000901A1968B8EE612AC1F3080101EE901AF6
:10184000F8EE611A40EE201A31EE810A22EE000A0B
:10185000A2E700E013E0B4FBF1F101EE901A196881
:10186000B8EE612AC1F3080101EE901AF8EE611A90
:1018700040EE201A31EE810A22EE000A8CE70E4A71
:10188000B2FBF1F101EE901A1968B8EE612AC1F3CA
:10189000080101EE901AF8EE611A40EE201A31EEBE
:1018A000810A22EE000A77E7284402580000003936
:1018B00000093D000090D00340787D012DE9F84FEC
:1018C000044600250026FB4F2068DFF8EC83010169
:1018D00004F1240000900DD5606EB0B1B0F5801F0A
:1018E00018D0B0F5001F1BD0B0F5401F00D0012567
:1018F000E5B12E462088C00535D5606D05282FD26C
:10190000DFE800F01D22282F2F00386840F4003057
:101910003860EDE70221201D02F03CFA0546E7E7BA
:101920000098022102F0B6FA0546E1E7D8F8000077
:10193000616E20F440100843C8F80000DAE7386808
:1019400040F4003038600CE00021201D02F022FA43
:10195000054606E00098002102F09CFA054600E0EA
:1019600001255DB12E432088800518D5A06D802803
:1019700030D00CDC18B340280ED125E0D8F8000098
:10198000616D20F007000843C8F80000EBE7C028AD
:1019900003D0B0F5807F00D001250DB32E43208801
:1019A000DFF8189340052DD5D4F8A400B0F5800FCA
:1019B00042D01EDCA0B3B0F5001F20D136E038685D
:1019C00040F400303860E8E70021201D02F0E2F921
:1019D0000546E2E70098002102F05CFA0546DCE7E4
:1019E000D8F80000A16D20F4E0700843C8F80000AA
:1019F000D5E7B0F5C00F03D0B0F5000F00D001253A
:101A000005B32E43208800052FD5D4F8A800B0F1E7
:101A1000007F52D020DCE8B3B0F1807F22D146E0D5
:101A2000FFE7386840F400303860E9E70021201D06
:101A300002F0B0F90546E3E70098002102F02AFA27
:101A40000546DDE7D9F80000D4F8A41020F46000C2
:101A50000843C9F80000D5E7B0F1407F03D0B0F1EA
:101A6000806F00D0012575B32E43206880010AD510
:101A7000A06C30B1102831D0202835D0302800D0CB
:101A8000012585B32E432088C00446D5E06DB0F50E
:101A9000005F00E006E05BD036DCA0B3B0F5805F0D
:101AA00038D14FE0386840F400303860DBE700217F
:101AB000201D02F06FF90546D5E70098002102F0DD
:101AC000E9F90546CFE7FFE7D9F80000D4F8A810F8
:101AD00020F0E0600843C9F80000C6E7386840F429
:101AE00000303860CDE705E00221201D02F052F9F8
:101AF0000546C6E77048001F0168A26C21F030015E
:101B000011430160BFE718E0B0F5405F03D0B0F5C6
:101B1000804F00D001250DB32E43208880042FD59F
:101B2000206EB0F5403F29D021DC38B3B0F5803FBE
:101B300037D0B0F5003F20D139E0386840F40030AC
:101B40003860E8E70021201D02F024F90546E2E7AD
:101B50000098002102F09EF90546DCE7D8F8000065
:101B6000E16D20F4E0400843C8F80000D5E7B0F587
:101B7000802F03D0B0F5A02F00D00125EDB12E436A
:101B8000208840042BD5D4F8AC00B0F1405F24D0BD
:101B90001CDC10B3B0F1805F4BD0B0F1005F1BD103
:101BA0004EE00121201D02F0F5F80546E6E7009819
:101BB000012102F06FF90546E0E7D8F80000216E38
:101BC00020F4E0200843C8F80000D9E7B0F1804FC6
:101BD00003D0B0F1A04F00D0012585B32E4320885B
:101BE00000040AD5E06E30B1B0F1805F39D0B0F1B9
:101BF000005F3BD001259DB32E432068C0010AD56C
:101C0000606C30B1012841D0022844D0032800D0B4
:101C100001258DB32E432068DFF8A4B0400261D5C2
:101C20002848016841F480710160FFF705FC824695
:101C300052E00121201D02F0ADF80546CDE705E098
:101C40000098012102F026F90546C6E7D9F8000000
:101C5000D4F8AC1020F0E0400843C9F80000BEE71B
:101C60000BE0386840F400303860C4E70121201DE3
:101C700002F090F80546BEE713E0D8F80000E16EE8
:101C800020F040500843C8F80000B6E7386840F438
:101C900000303860BDE70221201D02F07BF80546C8
:101CA000B7E70548001F0168626C21F0030111438A
:101CB0000160B0E72C44025850440258584402587E
:101CC0001044025800480258FFF7B6FBA0EB0A0088
:101CD000642801D9032503E0FE480068C005F3D558
:101CE0007DB12E432078DFF8F0A3C00766D0A06F47
:101CF000182861D05BDC80B308286AD010285AD13C
:101D00006DE0F5481C300068B4F8B01000F4407085
:101D100001F4407188420DD0EF481C30016821F475
:101D20004071026842F480320260026822F480321C
:101D300002600160D4F8B000B0F5807F13D1FFF7E6
:101D40007BFB82460AE0FFF777FBA0EB0A0141F23A
:101D50008830814202D9032505E02DE0DE481C30A1
:101D600000688007EFD50DB12E43BBE7D4F8B00073
:101D7000C0F3012103290FD0DBF8000020F47C50D0
:101D8000CBF80000D4481C300168B4F8B020C2F38E
:101D90000B0211430160A5E7DBF80010CF4A21F4E4
:101DA0007C51104041EA1010CBF80000EAE72028EF
:101DB00002D0282800D00125BDB12E43207880070D
:101DC0002BD5606F062825D2DFE800F025181E25E8
:101DD00025250121201D01F0DDFF0546ECE70098D7
:101DE000012102F057F80546E6E7DAF80000A16F96
:101DF00020F038000843CAF80000DFE70121201D69
:101E000001F0C8FF054606E00098012102F042F803
:101E1000054600E0012565B12E432078400720D516
:101E2000D4F89000062819D2DFE800F0190C121936
:101E30001919DAF80000616F20F007000843CAF8AA
:101E40000000EAE70121201D01F0A4FF054606E09D
:101E50000098012102F01EF8054600E001258DB131
:101E60002E432078800620D5D4F88C00B0F1405F56
:101E700019D011DCB8B1B0F1805F27D0B0F1005FAC
:101E800010D129E0D9F80000D4F8901020F0070014
:101E90000843C9F80000E4E7B0F1804F03D0B0F187
:101EA000A04F00D00125EDB12E43207840062CD55F
:101EB000D4F89800B0F5406F25D01DDC18B3B0F50C
:101EC000806F33D0B0F5006F1CD135E00021201DAC
:101ED00001F060FF0546E6E70098022101F0DAFF15
:101EE0000546E0E7DAF80000D4F88C1020F0E04076
:101EF0000843CAF80000D8E7B0F5805F03D0B0F51A
:101F0000A05F00D00125EDB12E43207800062CD52E
:101F1000D4F89C00B0F5C04F25D01DDC18B3B0F547
:101F2000005F7DD0B0F5804F1CD1DFE00021201D87
:101F300001F030FF0546E6E70098022101F0AAFF14
:101F40000546E0E7D9F80000D4F8981020F4E050F6
:101F50000843C9F80000D8E7B0F5004F03D0B0F54A
:101F6000204F00D00125EDB32E43207800070BD57C
:101F7000D4F88000B0F5805F76D0DAF8001021F454
:101F800040510143CAF800102078C0060BD5D4F8A0
:101F90009400B0F5807F69D0D9F8001021F4407129
:101FA0000143C9F80010206800030BD5D4F8A00045
:101FB000B8B3B0F5803F7ED0B0F5003F00D001252A
:101FC00085B32E43206840030FD5D4F88400B0F5C4
:101FD000801F71D0B0F5001F6FD0B0F5401F00D04A
:101FE000012500E088E0EDB32E432068C00307D54B
:101FF000E06CC0B3B0F5803F6BD00125ADB32E438C
:102000002068800004D50098022101F043FF0643B8
:102010002068800311D5E06F68B1B0F5807F02E0E1
:102020005EE080E08CE071D0B0F5007F03D0B0F5C9
:10203000407F00D00125EDB32E432068C00207D5B4
:10204000D8F80000216F20F000400843C8F80000D5
:102050002068C0000ED5DBF80000D4F8B41020F4DE
:10206000804004E081E08AE051E093E055E00843DD
:10207000CBF800002068800207D5D8F80000A16ED8
:1020800020F080700843C8F80000206840000CD59C
:10209000DBF8000020F40040CBF80000DBF8000083
:1020A000D4F8B8100843CBF80000206800280CDAF8
:1020B000094803E07BE03DE04CE050E0083801686F
:1020C000226D21F040511143016096B30120BDE81B
:1020D000F88F59E00048025854440258FFFCFF0FA3
:1020E0000021201D01F056FE05463CE70098022124
:1020F00001F0D0FE054636E7D9F80000D4F89C1070
:1021000020F460400843C9F800002EE74AE0009838
:10211000022101F0BFFE064336E70098022101F0DC
:10212000B9FE06433FE70021201D01F033FE0546BE
:1021300046E745E00098022101F0ACFE05463FE786
:10214000D9F80000D4F8A01020F440300843C9F8B2
:10215000000037E7386840F40030386041E7009805
:10216000012101F097FE05463BE7DAF80000D4F8BC
:10217000841020F440100843CAF8000035E738689E
:1021800040F40030386039E70221201D01F002FEE2
:10219000054633E70B480168E26C21F480311143B6
:1021A00001602DE7386840F40030386043E7DAF822
:1021B0000000E16F20F440700843CAF800003CE7DB
:1021C000002084E74C4402582DE9F04704460E46AF
:1021D000DFF8CC81D8F8000000F00700B0420FD241
:1021E000D8F8000020F007003043C8F80000D8F805
:1021F000000000F00700B04202D00120BDE8F087E7
:102200002078684F800705D53868E16820F00F0016
:10221000084338602078C00770D03868A16820F47F
:102220007060084338605F4960681839022808D038
:1022300003280BD001280ED00968490710D40120CB
:10224000DCE7096889030BD40120D7E70968890115
:1022500006D40120D2E70968C90501D40120CDE7E1
:10226000DFF84091A9F10809D9F8001021F0070121
:102270000143C9F80010FFF7DFF80546606841F236
:10228000883A02280BD0032817D0012823D030E049
:10229000FFF7D2F8401B504501D90320AEE7D9F82B
:1022A0000000C0F3C2000228F2D127E0FFF7C4F813
:1022B000401B504501D90320A0E7D9F80000C0F326
:1022C000C2000328F2D119E0FFF7B6F8401B5045D1
:1022D00001D9032092E7D9F80000C0F3C200012819
:1022E000F2D10BE0FFF7A8F8401B504501D90320BD
:1022F00084E7D9F8000010F0380FF3D1D8F80000C7
:1023000000F00700B0420ED9D8F8000020F0070016
:102310003043C8F80000D8F8000000F00700B042D1
:1023200001D001206AE72078400705D53868216987
:1023300020F070000843386020781B49000705D55D
:102340000868626920F07000104308602078C006B9
:1023500005D50868A26920F4E06010430860207881
:10236000800607D51049091D0868E26920F0700051
:102370001043086000F064F839684FF4807292FAF4
:10238000A2F201F47061B2FA82F2D140074A515CC4
:10239000C840074908600F20FFF76AF800202DE7C2
:1023A00000200052184402581C4402587C4F000878
:1023B0000000002410B5FFF7BDF8084909680122A4
:1023C00092FAA2F201F00F01B2FA82F2D140044A6D
:1023D000515CC8400349086010BD00001844025811
:1023E0007C4F00080400002410B5FFF7E3FF074905
:1023F0000968102292FAA2F201F07001B2FA82F298
:10240000D140034A515CC84010BD00001C44025832
:102410007C4F000810B5FFF7CDFF074909684FF45E
:10242000807292FAA2F201F4E061B2FA82F2D14033
:10243000024A515CC84010BD1C4402587C4F000841
:10244000F0B55C4800685D4D10F038015A4809D07D
:10245000041108290ED05A4E10290DD018290DD07C
:102460002046F0BD29688906FBD52968C1F3C10162
:10247000C840F0BD2046F0BD3046F0BD4D49183192
:102480000A6802F003020968C1F30511494B1C33C5
:102490001B6803F00103474F24373F68C7F3CC079D
:1024A00017FB03F300EE103AB8EE400ADFED450AE1
:1024B000404BB7EE001A20332AB3012A52D0022A29
:1024C00064D0B4FBF1F001EE900A1868B8EE612A0E
:1024D000C0F3080001EE900AF8EE611A40EE201AEF
:1024E00031EE810A22EE000A1868C0F34620401C33
:1024F00000EE900AF8EE600A80EE201ABCEEC10AE7
:1025000010EE100AF0BD2A68920617D52A68C2F3A9
:10251000C102D040B0FBF1F001EE900A1868B8EEAD
:10252000612AC0F3080001EE900AF8EE611A40EE4D
:10253000201A31EE810A22EE000AD5E7B0FBF1F055
:1025400001EE900A1868B8EE612AC0F3080001EEA7
:10255000900AF8EE611A40EE201A31EE810A22EE5E
:10256000000AC1E7B4FBF1F001EE900A1868B8EE7A
:10257000612AC0F3080001EE900AF8EE611A40EEFD
:10258000201A31EE810A22EE000AADE7B6FBF1F027
:1025900001EE900A1868B8EE612AC0F3080001EE57
:1025A000900AF8EE611A40EE201A31EE810A22EE0E
:1025B000000A99E7104402580090D00300440258E2
:1025C00040787D01000000392DE9F05F0446FC4FA2
:1025D000FC4E41F28838FC4D2078C0075FD0386847
:1025E000C0F3C20002281FD03868C0F3C20003281D
:1025F00004D1306800F00300022815D06068B0F5FF
:10260000803F19D0E8B1B0F5A02F23D0286820F47E
:1026100080302860286820F480202860606870B3CB
:10262000FEF70AFF814626E02868800337D56068F8
:1026300020BB0120BDE8F09F286840F4803028606E
:10264000ECE7286820F480302860286820F4802097
:102650002860E3E7286840F480202860286840F478
:1026600080302860DAE7FEF7E7FEA0EB090040457E
:1026700001D90320DEE728688003F4D50FE0FFE7E7
:10268000FEF7DAFE814607E0FEF7D6FEA0EB090072
:10269000404501D90320CDE728688003F4D4207891
:1026A000DFF828A380076FD538684FF47C3B10F023
:1026B000380F12D03868C0F3C200032802D1306846
:1026C00080070AD0E06890B3296821F0190101431E
:1026D0002960FEF7B1FE814632E02868400701D547
:1026E000E06848B12868E16820F0190008432860D4
:1026F000FEF7A2FE814609E001209BE7FEF79CFE63
:10270000A0EB0900022801D9032093E728684007BD
:10271000F4D5DAF800009BFAABF22169B2FA82F242
:1027200020F47C3091400843CAF800002CE018E007
:10273000FEF782FEA0EB0900022801D9032079E709
:1027400028684007F4D5DAF800009BFAABF220F4D1
:102750007C312069B2FA82F290400143CAF800103D
:1027600012E0286820F001002860FEF765FE81462F
:1027700007E0FEF761FEA0EB0900022801D9032063
:1027800058E728684007F4D42078C0065DD538683B
:102790004FF0F84BC0F3C200012813D03868C0F3E3
:1027A000C200032804D1306800F00300012809D0DA
:1027B000E069B0B3286840F080002860FEF73CFE76
:1027C00081461DE02868C00504D5E069802801D055
:1027D00001202FE7DAF800009BFAABF220F0F84175
:1027E000206AB2FA82F290400143CAF800102CE04D
:1027F000FEF722FEA0EB0900022801D9032019E709
:102800002868C005F4D5DAF800009BFAABF2216A1B
:10281000B2FA82F220F0F84091400843CAF8000072
:1028200013E0FFE7286820F080002860FEF704FE30
:10283000814607E0FEF700FEA0EB0900022801D95F
:102840000320F7E62868C005F4D42078000732D5C5
:10285000DFF870A160690AF14C0AB0B1DAF8000043
:1028600040F00100CAF80000FEF7E6FD814607E0EF
:10287000FEF7E2FDA0EB0900022801D90320D9E60A
:10288000DAF800008007F3D515E0DAF8000020F050
:102890000100CAF80000FEF7CFFD814607E0FEF711
:1028A000CBFDA0EB0900022801D90320C2E6DAF82B
:1028B00000008007F3D42078800628D5A06998B15D
:1028C000286840F480502860FEF7B6FD814607E096
:1028D000FEF7B2FDA0EB0900022801D90320A9E60A
:1028E00028688004F4D512E0286820F4805028601D
:1028F000FEF7A2FD814607E0FEF79EFDA0EB090072
:10290000022801D9032095E628688004F4D42078B1
:1029100040077CD5DFF8B8A0DAF8000040F48070FA
:10292000CAF80000FEF788FD814607E0FEF784FD47
:10293000A0EB0900642801D903207BE6DAF8000047
:10294000C005F3D5DFF87C90A06809F1480901289B
:1029500014D0D0B1052825D0D9F8000020F001000E
:10296000C9F80000D9F8000020F00400C9F8000000
:10297000A06820B3FEF760FD824633E0D9F800007E
:1029800040F00100C9F80000F2E7D9F8000020F09B
:102990000100C9F80000D9F8000020F00400C9F8CF
:1029A0000000E5E7D9F8000040F00400C9F8000095
:1029B000D9F8000040F00100C9F80000D8E716E09F
:1029C0001044025828440258004402580444025853
:1029D00000480258FEF730FDA0EB0A00404501D93F
:1029E000032027E6D9F800008007F3D50FE0FEF7B3
:1029F00023FD824607E0FEF71FFDA0EB0A004045DD
:102A000001D9032016E6D9F800008007F3D4606AE4
:102A1000E8B33968C1F3C201032975D0022807D091
:102A2000286820F080702860FEF706FD04467EE0EE
:102A3000286820F080702860FEF7FEFC074606E05C
:102A4000FEF7FAFCC01B022801D90320F2E5286832
:102A50008001F5D4306840F2F3318843E16A40EAFE
:102A60000110A16A08433060208E4FF6FF72616B3F
:102A7000401E491EC0F3080002EA41210843218F8D
:102A80004FF4FE02491E02EA0141084300E051E012
:102A900094F83C10491E120202EA016108432749DA
:102AA0000860091D08684FF6F872A36C904392FA0B
:102AB000A2F2B2FA82F29340184308601F48001F46
:102AC0000168226C21F00C01114301600168626C05
:102AD00021F0020111430160016841F4803101607D
:102AE000016841F400310160016841F48021016016
:102AF000016841F001010160286840F080702860A1
:102B0000FEF79AFC044607E016E0FEF795FC001B72
:102B1000022801D903208DE528688001F5D509E058
:102B2000FEF78AFC001B022801D9032082E52868F1
:102B30008001F5D400207DE501207BE5304402587A
:102B40002DE9F05F04460025002C12D04FF4800BD5
:102B5000DFF8D8812068764E764F40450BD0B042E2
:102B600009D0B84207D0E0680F2804D90120BDE899
:102B7000F09F0120FBE7204601F0CEFA01462068D5
:102B8000404505D0B04203D0B84201D0082907D84B
:102B9000404503D0B04201D0B84203D1102901D939
:102BA0000120E4E7A16A4FF4702A594514D1404549
:102BB00008D0B04206D0B84204D0206B504501D9AD
:102BC0000120D4E7256B0DB9A0890504E068B0EBBE
:102BD000154F01D90120CAE794F881004FF0000990
:102BE00020B984F88090204600F0A6F8022084F8EE
:102BF00081002068016821F001010160A069B0F145
:102C0000806F09D16068584506D1A06B20B9206853
:102C1000016841F480510160A16AE0690843E16BF9
:102C200029430843E168084321688860616A606B52
:102C3000A2690843A16B11430843216908436169F4
:102C40000843216A084361680843E16C0843A168AE
:102C50000843A16C0843A16D08432168C860A06ABD
:102C6000584528D1206C012828D02068016821F41B
:102C700000410160606C012826D02068016821F4C1
:102C8000804101602068404505D0B04203D0B84281
:102C900001D055451ED0404503D0B04201D0B842C6
:102CA00002D1B5F5F81F15D0016821F4005101607B
:102CB0002168E06A0864606888B120E020680168E3
:102CC00041F400410160D5E72068016841F480418A
:102CD0000160D7E7016841F400510160E8E7A06AAC
:102CE00030B92068816821F4C05141F400618160ED
:102CF0002068816821F4C06141F4806181602068AE
:102D0000016D21F0010101656068400206D520686F
:102D1000C168626D21F000411143C160C4F8849024
:102D2000012084F88100002021E7000000300140EC
:102D300000380040003C004000B5B5B015480168BF
:102D400041F002010160006800F0020000901148AB
:102D50000830016841F480410160006800F480405F
:102D600000904FF4805001900020189001A8FEF7C9
:102D7000A5FD4FF460403090022031900120329048
:102D80000320339005203490034830A9FEF754FA0D
:102D900035B000BDE0440258000402582DE9F84F58
:102DA00004468A46934699460A9D94F88000012875
:102DB00013D04FF0010884F88080FEF73DFB0646F3
:102DC00094F88100002701284FF4800110D060683A
:102DD000884209D1A06838B902E00220BDE8F88F26
:102DE00094F88100042803D0022084F88070F5E76D
:102DF000BAF1000F34D0BBF1000F31D0B9F1000FA0
:102E00002ED094F88100042802D0052084F8810097
:102E1000C4F88470C4F864B0A4F86A90A4F8689008
:102E2000C4F85CA0A4F86290A4F860902767676774
:102E3000206842686FF30F0242EA0902426020688C
:102E4000026842F0010202606068884204D1206892
:102E5000016841F400710160E0680F283ED846E047
:102E6000012084F88070B9E7B4F8620070B120687E
:102E7000416989070AD5E16D09680162E06D001DAD
:102E8000E065B4F86200401EA4F86200B4F86A007D
:102E900080B12068416948F2080211420AD0006BF3
:102EA000616E0860606E001D6066B4F86A00401EC6
:102EB000A4F86A00681C11D0FEF7BEFA801BA84275
:102EC0000CD3204601F0BAF804F8807F606840F423
:102ED0008070606084F8018001207FE7B4F86200B0
:102EE0000028C1D1B4F86A000028BDD1EFE007285E
:102EF0005AD8E3E0B4F8620000B32068416989075A
:102F00001CD5B4F8621001290DD9E16B59B1E16DFE
:102F100009680162E06D001DE065B4F86200801E82
:102F2000A4F862000AE0E16D09880184E06D801C6C
:102F3000E065B4F86200401EA4F86200B4F86A00CC
:102F4000F0B12068416911F4604F19D0416909045A
:102F50000BD5006B616E0860606E001D6066B4F892
:102F60006A00801EA4F86A000AE0008E616E088084
:102F7000606E801C6066B4F86A00401EA4F86A00A7
:102F8000681C11D0FEF758FA801BA8420CD32046CB
:102F900001F054F804F8807F606840F4807060604D
:102FA00084F80180012019E7B4F862000028A1D15B
:102FB000B4F86A0000289DD189E0B4F8620038B303
:102FC00020684169890730D5B4F8621003290ED909
:102FD000E16B40290BD9E16D09680162E06D001DCC
:102FE000E065B4F86200001FA4F862001DE0B4F8C8
:102FF000621001290DD9E16B59B1E16D0988018495
:10300000E06D801CE065B4F86200801EA4F86200E8
:103010000BE0E16D097880F82010E06D401CE06560
:10302000B4F86200401EA4F86200B4F86A0020B34D
:103030002068416911F4604F2CD0416909040BD517
:10304000006B616E0860606E001D6066B4F86A0017
:10305000001FA4F86A001DE0416901F4C041B1F508
:10306000005F0BD9008E616E0880606E801C606608
:10307000B4F86A00801EA4F86A000BE090F83000F3
:10308000616E0870606E401C6066B4F86A00401E95
:10309000A4F86A00681C11D0FEF7CEF9801BA84284
:1030A0000CD3204600F0CAFF04F8807F606840F42B
:1030B0008070606084F8018001208FE6B4F86200BF
:1030C00000287FF47AAFB4F86A000028F9D1002212
:1030D000334608212046009501F028F828B1D4F89D
:1030E000840040F02000C4F88400204600F0A6FFD1
:1030F00004F8807F84F80180606808B101206DE6E3
:1031000000206BE604284FF0E02104D0086920F08D
:10311000040008617047086940F0040008617047C6
:1031200010B5401EB0F1807F01D3012010BD4FF0DB
:10313000E02460610F21601701F083FE0020A06190
:1031400007202061002010BD70477047014611F82C
:10315000790F4978084370472DE9F0410446236808
:10316000D8691A68996800F00F05002D0CD1860601
:103170000AD502F0200601F080573E4304D02046D5
:10318000BDE8F04101F0F5B9002D74D0524D02F4C4
:1031900090760D4035436ED0C50707D0D50505D5CF
:1031A00001251D62E36F43F00103E367830708D540
:1031B000CB0706D0256802232B62E36F43F004039C
:1031C000E367430708D5CB0706D0256804232B62A5
:1031D000E36F43F00203E36703070ED502F0200319
:1031E00001F080552B4301D1CB0706D02568082379
:1031F0002B62E36F43F00803E367E36F002B2DD0EE
:10320000800608D502F0200001F08051084302D06A
:10321000204601F0AEF9E06F000703D42068806813
:10322000400621D5204601F089F9206881684906C9
:1032300016D5816821F040018160606F58B127493F
:103240000165606FFDF79CFF002807D0606F016D7E
:10325000BDE8F04108472046FFF777FFBDE8F08161
:103260002046FFF772FFF9E72046FFF76EFF0020C8
:10327000E067F3E7FFE7C5020ED54D020CD54FF42A
:1032800080101862202084F8790084F87A002046A3
:10329000BDE8F041FFF758BF05060AD502F08005EA
:1032A00001F400010D4304D02046BDE8F04101F0D7
:1032B00038BD410606D5510604D52046BDE8F0418B
:1032C00001F04AB90002C9D55000C7D5186820F0EE
:1032D00080401860C2E70000010000102945000886
:1032E00010B50446002C03D094F8790010B107E023
:1032F000012010BD002084F87800204600F028F856
:10330000242084F879002068016821F0010101601F
:10331000204601F06BF9012818D0606B10B12046EF
:1033200001F070F82068416821F490414160206804
:10333000816821F02A0181602068016841F0010163
:1033400001602046BDE8104001F0C0B8012010BD6A
:1033500010B586B000681B49884230D11A48016810
:1033600041F001010160006800F001000090164882
:103370001030016841F010010160006800F0100099
:1033800000904FF4007001900220029001210391FF
:1033900004900720059001A90C4C2046FDF74CFF36
:1033A0004FF48061019101A92046FDF745FF2520DA
:1033B000FEF781F8032225201146FEF789F806B0B2
:1033C00010BD000000100140E04402580000025807
:1033D00090F87A30202B01D002207047B9B1B2B1F9
:1033E00090F87830012B14D0012380F878304166B2
:1033F000A0F86820A0F86A20FF228168B1F5805FFC
:1034000009D07F2389B1B1F1805F16D01AE0012085
:10341000704702207047016911B1A0F86C2011E0DB
:1034200040F2FF11A0F86C100CE0016911B1A0F896
:103430006C3007E0A0F86C2004E00169E1B13F21A5
:10344000A0F86C100021C167222280F87A2080F851
:10345000781001688A6842F001028A6001680A688F
:1034600092000CD50A6842F480720A600068816894
:1034700041F08051816006E0A0F86C30E2E7086816
:1034800040F49070086000207047000030B500687C
:10349000124988420CD1124A5088010408D41146BE
:1034A0004FF000034404097807D50A2901D053805E
:1034B00030BD40F40040508030BD0D290AD0094D88
:1034C000C0F30D042955401C80B25080C728F3D9A1
:1034D000538030BD40F48040508030BD001001402A
:1034E0000C000024240000247047FEE72DE9F04181
:1034F000074600240C4E002108467388328800F0ED
:1035000023FB3588708845430021084600F008FBFE
:1035100000F00CFC03E0384600F0B2FB641CAC4247
:10352000F9D3BDE8F0810000F40100242DE9F04159
:103530002A4D0027F0212C232A242B2600284FF483
:10354000A07229D001282FD002284FF0010C33D0CF
:1035500003283AD0AF7129806A802B816C81AE81BB
:103560000024688900F0C6FB002000F089FB288851
:10357000401E80B200F084FBA88900F0BBFB002055
:1035800000F07EFB6888401E80B200F079FB204688
:10359000BDE8F04100F0A8BAAF7129806A802B81A4
:1035A0006C81AE810024DCE7AF7129806A802B81B9
:1035B0006C81AE810324D4E785F806C02A80698037
:1035C0002B816C81AE810524CBE785F806C02A806B
:1035D00069802B816C81AE810624C2E7F40100244E
:1035E0002DE9FE4F00250026171AA3EB010881469E
:1035F0008A46681E002F03DD4FF00101019107E0AC
:1036000003D14FF00001019102E00190C7F10007E2
:10361000B8F1000F03DD4FF00100009007E003D187
:103620004FF00000009002E00090C8F1000847450C
:1036300001DD3C4600E044464FF0000B601C029068
:1036400016E01FFA8AF10C9A1FFA89F000F09EF832
:103650003D444644A54202DD2D1B01988144A6420B
:1036600002DD361B009882440BF1010B1FFA8BFB25
:1036700002988345E5DDBDE8FE8F2DE9F8438046DD
:103680000E4615461F46089C33462A46314640469C
:103690000094FFF7A5FF3B46424631464046009462
:1036A000FFF79EFF3B462A46394640460094FFF707
:1036B00097FF3B462A46314628460094FFF790FF85
:1036C000BDE8F8832DE9FF4F83B007468846002404
:1036D00015460320A0EB420653E0A8EB0500069A2E
:1036E00081B2029007EB040A1FFA8AF000F04EF84C
:1036F000A8EB0400019081B2069A07EB05091FFAB6
:1037000089F000F043F808EB040B069A1FFA8BF1DE
:103710001FFA89F000F03AF808EB0509069A1FFA3B
:1037200089F11FFA8AF000F031F81FFA89F1069A40
:10373000A7EB04091FFA89F000F028F8A7EB050AA7
:10374000069A1FFA8BF11FFA8AF000F01FF8029810
:10375000069A81B21FFA89F000F018F80198069ACB
:1037600081B21FFA8AF000F011F8641C002E03DA0F
:1037700006EB8406B61D04E0601B06EB80060A36E5
:103780006D1EAC42A9DD07B0BDE8F08F2DE9F04118
:1037900007460E4615460A4C608900F0ABFA3846DB
:1037A00000F06EFAA08900F0A5FA304600F068FA41
:1037B000208900F09FFA2846BDE8F04100F060BA89
:1037C000F40100242DE9F0478146884615461C4641
:1037D000089F1F4E708900F08DFA484600F050FA9D
:1037E000681E80B200F04CFAB08900F083FA4046BF
:1037F00000F046FA601E80B200F042FA308900F014
:1038000079FAA5EB0905A4EB0800454300F08EFA10
:10381000002403E0384600F033FA641CAC42F9D9C6
:10382000708900F067FA002000F02AFA3088401E04
:1038300080B200F025FAB08900F05CFA002000F0B8
:103840001FFA7088BDE8F047401E80B200F018BA39
:10385000F401002410B586B01948016841F0020156
:103860000160006800F00200009041F20300019046
:103870000120029003900320049001A9114C2046DE
:10388000FDF7DAFC012220461146FDF7CFFD0122AB
:1038900020460221FDF7CAFD012220461103FDF753
:1038A000C5FD00F077FBA00400F0B0FB00F00CF8C1
:1038B000012220461146FDF7B9FD06B010BD0000FB
:1038C000E0440258000402587047000010B5FFF7AA
:1038D000C1FF00F0CBF9322001F0DCFACF2000F07C
:1038E00009FA002000F0EAF9D92000F0E7F93020C9
:1038F00000F0E4F9ED2000F0FDF9642000F0DEF9BD
:10390000032000F0DBF9122000F0D8F9812000F04C
:10391000D5F9E82000F0EEF9852000F0CFF910206D
:1039200000F0CCF9782000F0C9F9CB2000F0E2F9E2
:10393000392000F0C3F92C2000F0C0F9002000F07D
:10394000BDF9342000F0BAF9022000F0B7F9F720F1
:1039500000F0D0F9202000F0B1F9EA2000F0CAF917
:10396000002000F0ABF9002000F0A8F9C02000F022
:10397000C1F9212000F0A2F9C12000F0BBF912200A
:1039800000F09CF9C52000F0B5F9322000F096F95E
:103990003C2000F093F9C72000F0ACF9C12000F002
:1039A0008DF9362000F0A6F9082000F087F93A20BA
:1039B00000F0A0F9552000F081F9B12000F09AF94B
:1039C000002000F07BF9182000F078F9B62000F014
:1039D00091F90A2000F072F9A22000F06FF9F220AC
:1039E00000F088F9002000F069F9262000F082F943
:1039F000012000F063F9E02000F07CF90F2000F0D6
:103A00005DF9202000F05AF91E2000F057F9092036
:103A100000F054F9122000F051F90B2000F04EF99B
:103A2000502000F04BF9BA2000F048F9442000F093
:103A300045F9092000F042F9142000F03FF9052073
:103A400000F03CF9232000F039F9212000F036F98C
:103A5000002000F033F9E12000F04CF9002000F0E4
:103A60002DF9192000F02AF9192000F027F900207B
:103A700000F024F9122000F021F9072000F01EF9CF
:103A80002D2000F01BF9282000F018F93F2000F04D
:103A900015F9022000F012F90A2000F00FF90820B1
:103AA00000F00CF9252000F009F92D2000F006F9AE
:103AB0000F2000F003F9112000F01CF9782001F02C
:103AC000E9F9292000F016F90020FFF72FFD012267
:103AD00004481146FDF7AAFCBDE810404FF6FF7000
:103AE000FFF704BD000402580021082812D2DFE8C5
:103AF00000F0110406080A0C0E1080210AE0402193
:103B000008E0C02106E0202104E0602102E0A021BD
:103B100000E0E021362041F0080100F00DB900007E
:103B200070B506460D46074C608900F0E3F8304654
:103B300000F0A6F8A08900F0DDF82846BDE8704046
:103B400000F09EB8F40100242DE9F04105460C4632
:103B5000A818401E86B2E018401E87B2DFF82C80FD
:103B6000B8F80A0000F0C6F8284600F089F8304698
:103B700000F086F8B8F80C0000F0BCF8204600F021
:103B80007FF83846BDE8F04100F07AB8F40100242F
:103B90002DE9F84F82460C461F46A346780701D010
:103BA000012000E00020790800EBD7004843C0B2B4
:103BB0000090203A02F0FF09002648E00C2F13D0B5
:103BC000102F18D0182F45D1234909EBC90001EB5C
:103BD0008000855D4FF00008280611D50A9A21461D
:103BE0005046FFF7D3FD13E01C4909EB490001EBF8
:103BF0008000855DEEE71A4800EB0910855DE9E776
:103C00000B9828B91748214642885046FFF7BEFD59
:103C10006806050E641CA4B213484088A04219D956
:103C2000A4EB0B00B84209D15C460AF1010A1FFA65
:103C30008AFA0D48008850450CD906E008F10108C1
:103C400008F0FF08B8F1080FC6D3761CF6B200984A
:103C50008642B3D3BDE8F88F085A0008A44F000885
:103C6000185400081C000024F401002410B50120A1
:103C700000F040F8BDE81040322001F00BB9000020
:103C800070B504460C4E4FF480550022294630464C
:103C9000FDF7CCFB012230460221FDF7C7FB200ACD
:103CA00000F0A4F9E0B200F0A1F929463046BDE8E1
:103CB00070400122FDF7BABB0004025870B50646F9
:103CC0000B4D4FF48054002221462846FDF7AEFBF1
:103CD000012228460221FDF7A9FB304600F086F9B3
:103CE00021462846BDE870400122FDF79FBB000039
:103CF0000004025870B504460B4E4FF48055002264
:103D000029463046FDF792FB002230460221FDF79E
:103D10008DFBE0B200F06AF929463046BDE87040FC
:103D20000122FDF783BB000000040258014800890E
:103D3000FFF7E0BFF401002410B50C46FFF7DAFFEF
:103D4000E0B2BDE81040FFF7B9BF000010B586B083
:103D50000D48016841F001010160006800F00100B8
:103D60000090022001900120029003900320049013
:103D700001A9064C2046FDF75FFA012220460221E8
:103D8000FDF754FB06B010BDE04402580000025895
:103D9000704770472DE9F047044688460027DFF852
:103DA000F090D9F80000C043800709D0384D283D75
:103DB000286820F080602860FDF73EFB064609E099
:103DC0000120BDE8F087FDF737FB801B022801D9F1
:103DD0000320F6E728680001F5D4D9F8000021682F
:103DE00020F47C3040EA0130C9F80000A0884FF68A
:103DF000FF72A168401E491EC0F3080002EA41217B
:103E00000843A1894FF4FE02491E02EA014108431A
:103E1000217C1202491E02EA016108431C4910314B
:103E200008601B48001D0168626921F0C001114350
:103E300001600168A26921F0200111430160B8F11D
:103E4000000F0ED0B8F1010F10D0016841F400113D
:103E50000160286840F080602860FDF7EDFA0446B4
:103E600010E0016841F400210160F2E7016841F4CB
:103E700080110160EDE7FDF7DFFA001B022801D990
:103E800003209EE728680001F5D5384699E7000031
:103E9000284402582DE9F047044688460027DFF8F9
:103EA000F090D9F80000C043800709D0384D283D74
:103EB000286820F080502860FDF7BEFA064609E029
:103EC0000120BDE8F087FDF7B7FA801B022801D971
:103ED0000320F6E728688000F5D4D9F8000021888F
:103EE00020F07C7040EA0150C9F80000A0884FF62D
:103EF000FF72A168401E491EC0F3080002EA41217A
:103F00000843A1894FF4FE02491E02EA0141084319
:103F1000217C1202491E02EA016108431C49183142
:103F200008601B48001D0168626921F4406111436B
:103F300001600168A26921F4007111430160B8F1C8
:103F4000000F0ED0B8F1010F10D0016841F0807160
:103F50000160286840F080502860FDF76DFA044643
:103F600010E0016841F480010160F2E7016841F46A
:103F700000010160EDE7FDF75FFA001B022801D99F
:103F800003209EE728688000F5D5384699E70000B1
:103F90002844025810B5144C124820604FF4800099
:103FA00060600020A0600721E1604FF00072226194
:103FB000521062619200A2616063CA0762650A07DB
:103FC000E26120626062A062E1622046FEF7B8FD15
:103FD0002068016841F001010160BDE81040FF2048
:103FE00000F004B8003800406C01002401B582B034
:103FF0004FF47A700123009001AA034802A9FEF74A
:10400000CDFE9DF804000EBD6C0100240A4A116823
:104010000B6823F001030B6011688B6823F0E04309
:104020008B6011688B6803438B601068016841F0F6
:1040300001010160704700006C01002410B50268A6
:104040005169936943F0080393610268936943F0EF
:10405000100393610268136823F001031360026880
:10406000136940F26B34A34313610268936823F42D
:104070004043936090F88120042A0CD08A060AD528
:10408000D0F8842042F08002C0F88420026893694E
:1040900043F02003936190F88120032A1DD04A0643
:1040A0000AD5D0F8842042F00402C0F884200268C7
:1040B000936943F040039361826AB2F5800F0CD19B
:1040C0000A060AD5D0F8842042F00202C0F8842003
:1040D0000268936943F0800393618A050AD5D0F89A
:1040E000842042F00102C0F884200268936943F4FE
:1040F00000739361C9050AD5D0F8841041F0080116
:10410000C0F8841001688A6942F480728A610021D3
:1041100020F8621F018110BDC16B012202EB511119
:10412000C068401CC01DC008484370472DE9F041DD
:1041300006460D4617469846069C0BE0601C09D0C3
:104140002CB1FDF779F9A0EB0800A04202D90320B9
:10415000BDE8F0813068406935EA000004D00020F5
:10416000B842EBD00020F3E70120F9E770470000E8
:104170002DE9F04F93B004468A4615461F46A146E6
:10418000780701D0012000E0002000EBD700784341
:10419000C0B200900C2F03D0102F01D0182F36D1B1
:1041A000009A01A93B462846FCF7C2FF4FF00008E1
:1041B0002AE001A810F808600025DFF858B03006A2
:1041C00005D51C9A51462046FFF7E0FA07E01D98F6
:1041D00028B9BBF8002051462046FFF7D7FA7006F1
:1041E000060E641CA4B2A4EB0900B84204D14C46EC
:1041F0000AF1010A1FFA8AFA6D1CEDB2082DDED30E
:1042000008F1010808F0FF0800988045D1D313B0E9
:10421000BDE8F08F1E0000242DE9FF4F83B0044657
:104220000E469346DDE91075A046B2464FF00009F0
:104230001EE0B9F1000F21D04FF0000908EB0B0090
:10424000401BA04202DA701986B2444606985044D8
:10425000401BB0420FDBDDE912012B463A46CDE9A7
:10426000000131462046FFF783FFBF1C601984B26E
:104270003A78002ADDD107B0BDE8F08F802A02D954
:104280004FF00109F4E708EB0B00A0EB5500A0424A
:1042900002DA701986B2444606985044401BB04278
:1042A000E9DB0D2A0DD0DDE912012B46CDE9000135
:1042B00031462046FFF76CFC7F1C04EB550084B2AE
:1042C000D6E7701986B244467F1CF5E770B59CB0FE
:1042D000284C256825F0040525600026254C0C3463
:1042E000256845F440452560256805F4404500955E
:1042F0002568AD04FCD5012401942404029404969D
:10430000089602240A940B940D900C910E920F9330
:1043100012960824119401A8FEF756F910B1012055
:104320001CB070BD3F201490032015901696179472
:104330004020199001011A91189050201B900221E1
:1043400014A8FDF741FF08B10120E9E70A48016818
:1043500041F0800101600848F430016841F0020139
:104360000160006800F002000090FCF75DFF002093
:10437000D6E700000C48025800440258FDF762B826
:104380001C48016841F4700101601B49086840F055
:1043900001000860184A0020103210600A68174BAC
:1043A0001A400A60144A18321060121D1060121D63
:1043B0001060114A28321060121D1060121D10602A
:1043C000121D1060121D1060121D1060121D106071
:1043D000121D10600A6822F480220A6006496031CA
:1043E0000860012006490860C0060249803908605B
:1043F0007047000088ED00E0004402587FEDF6EAC7
:104400000881005190F83410C90706D001684A6845
:10441000836B22F400321A434A6090F83410890703
:1044200006D501684A68C36B22F480321A434A6099
:1044300090F83410490706D501684A68036C22F4E5
:1044400080221A434A6090F83410090706D50168A3
:104450004A68436C22F400421A434A6090F83410D0
:10446000C90606D501688A68836C22F480521A4313
:104470008A6090F83410890606D501688A68C36C92
:1044800022F400521A438A6090F83410490611D57C
:1044900001684A68036D22F480121A434A60016D74
:1044A000B1F5801F06D101684A68436D22F4C0024D
:1044B0001A434A6090F83410090606D501684A6824
:1044C000806D22F4002202434A607047F8B504462A
:1044D0000026E667FCF7B0FF0746206800686FF02B
:1044E0007E4500070AD500223B464FF400112046C6
:1044F000009500F050FC08B10320F8BD206800686A
:1045000040070AD500223B464FF480012046009523
:1045100000F041FC08B10320F8BD20207834607021
:10452000A07026700020F8BD10B5806B0021A0F8A7
:104530006A10A0F86210FEF708FE10BD01680A6854
:1045400022F490720A6001688A6822F001028A608F
:10455000202180F87A10704710B501680A6822F0AF
:1045600040020A60202180F87910FEF7BDFF00208C
:1045700010BD10B5B0F86C2090F87A300168222B8D
:1045800005D0088B40F008000883022010BD898CFC
:104590008368B3F5805F01D1036973B11140426E46
:1045A000531C43661170B0F86A10491E0904090CC7
:1045B000A0F86A1008D0002010BD436E1140198089
:1045C000416E891C4166EEE701680A6822F4907228
:1045D0000A6001688A6822F001028A60202180F85E
:1045E0007A10FEF753FF002010BD00002DE9F04FB8
:1045F00087B00446802500210027FD4B2068AE05CA
:10460000A26AD4F808C0D4F81080D4F81C904CEA00
:10461000080CD4F8148048EA09084CEA080C42EA6D
:104620000C02D0F800C0DFF8CC830CEA080C4CEA8E
:10463000020CC0F800C020684268D4F80CC022F414
:10464000405242EA0C024260A06922689A4203D0BA
:10465000D4F820C04CEA0000D4F828C0B44504D1F6
:10466000D4E90B6C46EA0C0630439668DFF888C341
:1046700006EA0C06064396602068C26A666A22F063
:104680000F023243C262DD4E2068DD4AB0421CD1C7
:10469000126802F03802182A11D005DC4AB1082A43
:1046A00009D0102A06D108E0202A0AD0282A01D1F0
:1046B00009E00125D8E00425D6E04025D4E008250E
:1046C000D2E01025D0E02025CEE0CE4EB04215D16C
:1046D000126802F00702062A05D2DFE802F003059D
:1046E00007090B0D0025BFE00425BDE04025BBE018
:1046F0000825B9E01025B7E02025B5E0C24EB0424C
:1047000015D1126802F00702062A05D2DFE802F08E
:10471000030507090B0D0025A6E00425A4E04025AC
:10472000A2E00825A0E010259EE020259CE0B74EE1
:10473000B04215D1126802F00702062A05D2DFE85E
:1047400002F0030507090B0D00258DE004258BE021
:10475000402589E0082587E0102585E0202583E0B5
:10476000AB4EB04215D1126802F00702062A7BD286
:10477000DFE802F0030507090B0D002574E00425AE
:1047800072E0402570E008256EE010256CE02025E1
:104790006AE0A04EB0421CD1126802F03802182A1A
:1047A00011D005DC4AB1082A09D0102A5CD108E0F2
:1047B000202A0AD0282A57D109E0012554E00425EF
:1047C00052E0402550E008254EE010254CE0202521
:1047D0004AE0914EB04215D1126802F00702062A53
:1047E00042D2DFE802F0030507090B0D00253BE08C
:1047F000042539E0402537E0082535E0102533E071
:10480000202531E0854EB04215D1126802F0070232
:10481000062A29D2DFE802F0030507090B0D00255F
:1048200022E0042520E040251EE008251CE010259C
:104830001AE0202518E0984216D1714A121D12681C
:1048400002F00702062A0FD2DFE802F0030507098B
:104850000B0D022508E0042506E0402504E00825AC
:1048600002E0102500E02025DFF8B891DFF890A1E4
:1048700098426B4E4FEA291BAAF1540A7ED10020C0
:10488000102D33D006DC022D16D0042D17D0082DA4
:1048900004D11EE0202D2BD0402D15D0012700285B
:1048A00009D0D4F8048008EB4801814202D8B0EB6B
:1048B000083F20D90127ACE1FCF756FEEFE704A83A
:1048C000FCF768FE0598EAE701A8FCF72DFF0298BF
:1048D000E5E7DAF80000800606D5DAF80000C0F354
:1048E000C10029FA00F0DAE74846D8E75846D6E78B
:1048F0004FF40040D3E729460025102975D006DC87
:10490000022911D0042924D0082904D151E02029FA
:104910006CD0402936D00127434AA0F5407191421E
:1049200065D82168C86074E1FCF71EFE626A002346
:10493000294636F81220FBF7CBFC62680902030215
:1049400041EA10615008181869410023FBF7C0FCC8
:10495000E2E704A8FCF71EFE616A0023059836F81A
:1049600011201946FBF7B4FC62680902030241EA10
:104970001061500818186941002300E09BE0FBF724
:10498000A7FCC9E701A8FCF7CFFE616A00230298E3
:1049900036F811201946FBF79BFC626809020302F6
:1049A00041EA10615008181869410023FBF790FC98
:1049B000B2E7DAF8000080063BD5DAF80000002301
:1049C000616AC0F3C10036F81120194629FA00F0D7
:1049D000FBF77EFC0902020241EA10614FEA58002F
:1049E000101842466941002320E037E04BE060E0C8
:1049F000000C0058F369FFCFFFF4FF1100100140D5
:104A0000544402580044004000480040004C00401C
:104A1000005000400014014000780040007C00403D
:104A20008C4F00080090D003FFFC0F00FBF750FCF8
:104A300072E7606A0023194636F810204846FBF7F3
:104A400047FC0902020241EA10614FEA58001018BF
:104A5000424669410023FBF73BFC5DE7606A0023A7
:104A6000194636F810205846FBF732FC09020202BC
:104A700041EA10614FEA580010184246694100238C
:104A8000FBF726FC48E7606A0023194636F8102039
:104A90004FF40040FBF71CFC0902020241EA1061DE
:104AA0004FEA58001018424669410023FBF710FCFA
:104AB00032E70127ADE0E3694FF4004293426ED143
:104AC000082D55D005DC9DB1012D20D0042D06D137
:104AD0002CE0102D73D0202D7ED0402D37D0012713
:104AE00021F00F00C1F3420108432168C86090E043
:104AF000FDF77AFC616A36F81110B0FBF1F0410065
:104B0000606801EB5001B1FBF0F081B2E8E7FDF71E
:104B100081FC616A36F81110B0FBF1F04100606869
:104B200001EB5001B1FBF0F081B2D9E704A8FCF72A
:104B300031FD616A059836F81110B0FBF1F04100C3
:104B4000606801EB5001B1FBF0F081B2C8E701A849
:104B5000FCF7EAFD616A029836F81110B0FBF1F03B
:104B60004100606801EB5001B1FBF0F081B2B7E7A2
:104B7000DAF80000800613D5DAF80000C0F3C100AF
:104B800029FA00F9606A36F81000B9FBF0F041002C
:104B9000606801EB5001B1FBF0F081B2A0E728E0C2
:104BA000606A36F81000B9FBF0F04100606801EB74
:104BB0005001B1FBF0F081B292E700E00CE0606AD6
:104BC00036F81000BBFBF0F04100606801EB5001CB
:104BD000B1FBF0F081B283E7606A36F81000B2FBF7
:104BE000F0F04100606801EB5001B1FBF0F081B2E0
:104BF00076E7082D55D005DC7DB1012D1DD0042DA3
:104C000006D12AE0102D72D0202D7DD0402D36D037
:104C1000012707B03846BDE8F08FFDF7E5FB616A74
:104C200036F81110B0FBF1F1606801EB5001B1FBF7
:104C3000F0F0216880B2C860EBE7FDF7EBFB616A3A
:104C400036F81110B0FBF1F1606801EB5001B1FBD7
:104C5000F0F0216880B2C860DBE704A8FCF79AFC9A
:104C6000616A059836F81110B0FBF1F1606801EB4C
:104C70005001B1FBF0F0216880B2C860C9E701A81B
:104C8000FCF752FD616A029836F81110B0FBF1F1A1
:104C9000606801EB5001B1FBF0F0216880B2C860A0
:104CA000B7E7DAF80010890612D5DAF80010C1F378
:104CB000C10129FA01F9616A36F81110B9FBF1F264
:104CC000616802EB5102B2FBF1F189B2C160A0E769
:104CD000616A36F81110B9FBF1F2616802EB51021A
:104CE000B2FBF1F189B2C16093E700E00CE0616AC8
:104CF00036F81110BBFBF1F2616802EB5102B2FB16
:104D0000F1F189B2C16084E7616A36F81110B2FB33
:104D1000F1F2616802EB5102B2FBF1F189B2C160BC
:104D200077E790F87910212901D002207047B0F878
:104D3000621021B18168B1F5805F14D015E001687F
:104D40000A68920004D58A6822F400028A6003E0AF
:104D50000A6822F080020A600068016841F04001A0
:104D6000016000207047016959B1C16D4A1CC265DC
:104D700002680978118530F8621F491E0180002001
:104D80007047C16D02680988C1F308011185C16DC2
:104D9000891CC165EFE72DE9F04104460E46174630
:104DA0009846069D1DE0681C1BD02DB1FCF744FB06
:104DB000A0EB0800A84214D92068016821F4D07142
:104DC00001602068816821F001018160202084F861
:104DD000790084F87A00002084F878000320BDE888
:104DE000F0812068C06936EA000004D00020B84293
:104DF000D9D00020F3E70120F9E7000070B50024C6
:104E00000C4D0D48FEF7A8F902E0641CAC4204D832
:104E10000948FEF79BF92028F7D1002402E0641C22
:104E2000AC4206D8054901220348FEF7D1FA002812
:104E3000F5D170BDFFFF0100EC0000240C00002440
:104E4000FEE70907090E002804DB00F1E02080F8E6
:104E50000014704700F00F0000F1E02080F8141DEE
:104E6000704702E008C8121F08C1002AFAD1704733
:104E70007047002001E001C1121F002AFBD17047DA
:104E800010B504460420FEF73DF90148046010BD4A
:104E90000800002470B5054600244FF47A7603E03C
:104EA000304600F005F8641CAC42F9D370BD000038
:104EB00070B500214FF0E0256C690A4A1268504332
:104EC000AB69AA699A42FCD003D2A3EB020319444E
:104ED00003E0A4EB02063344194413468142F0D3A5
:104EE00070BD000008000024FBF75EFAFCF7B2FA80
:104EF000042302220521A020FFF7E8F94FF4C8702F
:104F0000FFF7BEFF4FF4E13000F01CF8FEF71EFF84
:104F1000FEF7DCFCFBF782FF08494FF4784008807D
:104F20004FF47A75064CFBF74DFB02212046FCF747
:104F300079FA2846FFF7AEFFF5E700001C000024D1
:104F40000000025810B50B49094A0A604860002069
:104F50008860C860086188610C2048610846FEF7D7
:104F6000BFF9BDE81040044901220248FEF730BAFB
:104F700000100140EC0000240C00002400000000A0
:104F800001020304010203040607080901000200EC
:104F90000400060008000A000C0010002000400079
:104FA0008000000100000000000000000000000080
:104FB000000000003F400000000000000000300042
:104FC000400030004000000009000BC03D000BC055
:104FD0003D00090018C024407FE0224031800000DD
:104FE000180024C01B000D803240018003801C404B
:104FF00027401C80074000401000600000000000B7
:10500000000000000000000000001F802040402041
:105010000000402020401F80000000000900060022
:105020001F80060009000000040004003F80040007
:1050300004000000001000600000000000000000FC
:10504000040004000400040004000000000000400C
:105050000000000000000000002001C00600380031
:10506000400000001F802040204020401F800000A2
:10507000000010403FC000400000000018C0214068
:10508000224024401840000010802040244024404A
:105090001B80000002000D0011003FC00140000015
:1050A0003C80244024402440238000001F80244072
:1050B00024403440038000003000200027C0380026
:1050C000200000001B802440244024401B8000005E
:1050D0001C0022C0224022401F800000000000006F
:1050E0000840000000000000000000000460000014
:1050F00000000000000004000A0011002080404071
:1051000009000900090009000900000000004040F2
:10511000208011000A000400180020002340240011
:10512000180000001F802040274029401F40000039
:10513000004007C039000F0001C0004020403FC0C0
:10514000244024401B8000001F802040204020403D
:105150003080000020403FC0204020401F800000E1
:1051600020403FC024402E4030C0000020403FC0BF
:1051700024402E00300000000F001080204022400C
:105180003380020020403FC0040004003FC02040A4
:10519000204020403FC020402040000000602020F0
:1051A00020203FC02000200020403FC024400B00B2
:1051B00030C0204020403FC020400040004000C0A0
:1051C0003FC03C0003C03C003FC0000020403FC047
:1051D0000C4023003FC020001F8020402040204082
:1051E0001F80000020403FC0244024001800000021
:1051F0001F802140214020E01FA0000020403FC030
:105200002440260019C0004018C0244024402240F9
:1052100031800000300020403FC0204030000000BE
:1052200020003F80004000403F80200020003E00E2
:1052300001C0070038002000380007C03C0007C04C
:1052400038000000204039C0060039C0204000006E
:105250002000384007C0384020000000304021C006
:105260002640384020C00000000000007FE04020C1
:1052700040200000000070000C000380004000008F
:105280000000402040207FE00000000000002000DF
:10529000400020000000000000100010001000106E
:1052A000001000100000000040000000000000009E
:1052B000000002800540054003C0004020003FC0C0
:1052C00004400440038000000000038004400440C8
:1052D0000640000000000380044024403FC000401E
:1052E000000003800540054003400000000004402A
:1052F0001FC0244024402000000002E0055005505B
:105300000650042020403FC00440040003C0004079
:105310000000044027C00040000000000010001002
:10532000041027E00000000020403FC001400700BB
:1053300004C00440204020403FC000400040000026
:1053400007C0040007C0040003C00000044007C0F9
:105350000440040003C000400000038004400440F7
:1053600003800000041007F0045004400380000094
:10537000000003800440045007F00010044007C000
:105380000240040004000000000006400540054003
:1053900004C00000000004001F8004400040000022
:1053A000040007800040044007C0004004000700DC
:1053B00004C0018006000400060001C0070001C00F
:1053C00006000000044006C0010006C004400000C2
:1053D0000410071004E001800600040000000440EF
:1053E00005C00640044000000000000004007BE00F
:1053F00040200000000000000000FFF0000000005E
:10540000000040207BE0040000000000400080001D
:1054100040002000200040000000000000000000CC
:1054200000000000000000000000000000001FCC91
:10543000000C0000000000000000080030006000C8
:105440000800300060000000022003FC1E20022043
:1054500003FC1E200220000000000E1811043FFF74
:1054600010840C78000000000F0010840F3800C07A
:10547000077818840078000000780F8410C4112485
:105480000E9800E400840008080068007000000026
:10549000000000000000000000000000000007E025
:1054A00018182004400200000000400220041818D0
:1054B00007E00000000000000240024001800FF001
:1054C00001800240024000000080008000800FF850
:1054D00000800080008000000001000D000E000030
:1054E000000000000000000000000080008000803C
:1054F00000800080008000800000000C000C000094
:10550000000000000000000000000006001800601D
:105510000180060018002000000007F008081004B1
:105520001004080807F000000000080408041FFC2D
:10553000000400040000000000000E0C10141024F1
:10554000104411840E0C000000000C18100411040B
:10555000110412880C700000000000E003200424F5
:1055600008241FFC0024000000001F981084110470
:105570001104108810700000000007F00888110462
:10558000110418880070000000001C00100010FCBE
:1055900013001C001000000000000E38114410849D
:1055A000108411440E38000000000700088C1044DD
:1055B0001044088807F00000000000000000030C01
:1055C000030C0000000000000000000000010106C4
:1055D00000000000000000000000008001400220E8
:1055E00004100808100400000220022002200220FB
:1055F000022002200220000000001004080804100D
:10560000022001400080000000000E001200100C7B
:10561000106C10800F00000003E00C1813E4142439
:1056200017C4082807D000000004003C03C41C4035
:10563000074000E4001C000410041FFC11041104C6
:1056400011040E880070000003E00C181004100410
:10565000100410081C10000010041FFC100410049B
:105660001004080807F0000010041FFC11041104C6
:1056700017C410040818000010041FFC11041100C6
:1056800017C010000800000003E00C1810041004FC
:1056900010441C780040000010041FFC108400809F
:1056A000008010841FFC10040000100410041FFC74
:1056B000100410040000000000030001100110019C
:1056C0001FFE10001000000010041FFC11040380D6
:1056D0001464181C1004000010041FFC10040004C3
:1056E00000040004000C000010041FFC1F0000FC5C
:1056F0001F001FFC1004000010041FFC0C0403001A
:1057000000E010181FFC100007F008081004100437
:105710001004080807F0000010041FFC108410801B
:10572000108010800F00000007F0081810241024CB
:10573000101C080A07F2000010041FFC11041100DD
:1057400011C011300E0C000400000E1C1104108456
:10575000108410441C3800001800100010041FFCB6
:10576000100410001800000010001FF810040004BE
:10577000000410041FF8100010001E0011E0001CAF
:10578000007013801C0010001FC0103C00E01F00C0
:1057900000E0103C1FC000001004180C163401C0BB
:1057A00001C01634180C100410001C00130400FC77
:1057B00013041C00100000000804101C1064108466
:1057C00013041C04101800000000000000007FFEFD
:1057D0004002400240020000000030000C00038044
:1057E0000060001C00030000000040024002400274
:1057F0007FFE0000000000000000000020004000CC
:1058000040004000200000000001000100010001F4
:1058100000010001000100010000400040002000E4
:105820000000000000000000000000980124014476
:105830000144014400FC000410001FFC0088010426
:10584000010400880070000000000070008801045E
:1058500001040104008800000000007000880104B9
:10586000010411081FFC0004000000F80144014479
:105870000144014400C800000000010401040FFCC1
:105880001104110411001800000000D6012901299B
:10589000012901C90106000010041FFC0084010059
:1058A0000100010400FC000400000104190419FCBB
:1058B00000040004000000000000000300010101DA
:1058C000190119FE0000000010041FFC0024004014
:1058D00001B4010C010400000000100410041FFCBE
:1058E0000004000400000000010401FC01040100A8
:1058F00001FC0104010000FC010401FC0084010022
:105900000100010400FC0004000000F8010401048F
:105910000104010400F80000010101FF00850104F9
:10592000010400880070000000000070008801047D
:105930000104010501FF00010104010401FC0084D0
:105940000104010001800000000000CC01240124BA
:10595000012401240198000000000100010007F863
:105960000104010400000000010001F8000400042B
:105970000004010801FC0004010001800170000C1A
:10598000001001600180010001F0010C003001C035
:105990000030010C01F0010000000104018C0074D2
:1059A0000170018C01040000010101810171000EF0
:1059B000001801600180010000000184010C013425
:1059C00001440184010C0000000000000000000000
:1059D00001003EFC40024002000000000000000008
:1059E000FFFF0000000000000000400240023EFCFB
:1059F0000100000000000000000060008000800046
:105A000040004000200020000000000000000000D6
:105A10000000000000000000000000000000000086
:105A20000000000000000000000000000000000076
:105A300000000000000000000000000F80380FFE92
:105A4000380F803800000000000000000000000057
:105A50000000000000000100000600000C000038FB
:105A600000003100000600000C000038000030008B
:105A7000000000000000000061800067F807F98066
:105A80000061800061800061800061800067F8072C
:105A9000F98000618000000000000000000001C0EB
:105AA000E003E0F00630080418081FFFFE040E08AB
:105AB0000787F00381E000000000000001F000060D
:105AC0000C00040408060C7001F9C0000E00003B35
:105AD000E000EC18070808040C180003E0000000C0
:105AE0000001E00007F003F818041C080417080779
:105AF000E1D003C0E00023B0003C08002008000013
:105B00001000000000000001000031000032000021
:105B10001C00000000000000000000000000000069
:105B20000000000000000000000000000000000075
:105B300000000000000000007F0001FFC00780F0AF
:105B40000C001810000420000200000000000020DB
:105B500000021000040C00180780F001FFC0007F55
:105B60000000000000000000000000000000000035
:105B7000000000004200006600006600003C0000DB
:105B8000180003FFC0001800003C0000660000661B
:105B900000004200000000000800000800000800AB
:105BA00000080000080001FFC00008000008000015
:105BB00008000008000008000000000000010000CC
:105BC0003100003200001C00000000000000000056
:105BD00000000000000000000000000000000000C5
:105BE0000800000800000800000800000800000885
:105BF0000000080000080000080000080000000085
:105C000000000000000000003800003800003800EC
:105C10000000000000000000000000000000000084
:105C20000000000000000000000600001C000070E2
:105C3000000180000E0000380000C0000700001CBA
:105C40000000300000000000000000007F8001FF25
:105C5000E00380700600180400080400080600181D
:105C600003807001FFE0007F800000000000000062
:105C7000000001000801000801000803FFF807FF09
:105C8000F800000800000800000800000000000004
:105C900000000001C03802C0580400980401180434
:105CA0000218040418061C1803F81801E0F8000094
:105CB0000000000000000001C0E003C0F004000884
:105CC00004080804080806180803F41801E7F0009F
:105CD00001E0000000000000000000000300000DD3
:105CE0000000110000610000810803010807FFF8AF
:105CF0000FFFF8000108000108000000000000008C
:105D000000E007FCD0060808061008061008061078
:105D100008061838060FF00607C000000000000053
:105D2000000000003F8001FFE003843002081804F7
:105D30001008041008041008071810030FF00007DB
:105D4000C000000000000000000003C000070000C9
:105D50000600000600F80607F806180006E000072F
:105D6000000006000000000000000001E1E003F771
:105D7000F0063410041808041808040C08040C0871
:105D800006161803F3F001C1E00000000000000057
:105D9000F80003FC30030638040208040208040279
:105DA000080404100308F001FFC0007F0000000099
:105DB00000000000000000000000000000000000E3
:105DC00070380070380070380000000000000000DB
:105DD00000000000000000000000000000000000C3
:105DE00000000000301A00301C000000000000001D
:105DF000000000000000000000000000000000089B
:105E000000001400002200004100008080010040DA
:105E1000020020040010080008000000000000003C
:105E200021000021000021000021000021000021AC
:105E300000002100002100002100002100000000DE
:105E4000000000000000080008040010020020010B
:105E50000040008080004100002200001400000883
:105E60000000000000000003C00004C000040000A7
:105E7000080038080F380808380810000C300007F0
:105E8000E00003C000000000000000003F8000FFB1
:105E9000E0038070020F1006708804C08804830835
:105EA000047F8802C09003012000FE40000008002B
:105EB00000180001F8003E0801C20007020007E2D6
:105EC0000000FE00001FC80001F8000038000008B4
:105ED00004000807FFF807FFF8040808040808048E
:105EE000080804080806180803F41801E7F0000180
:105EF000E0000000000000003F8001FFE003807030
:105F00000200180400080400080400080400100639
:105F100000200780C000000004000807FFF807FF0A
:105F2000F804000804000804000804001802001027
:105F300003807001FFE0007F80000000040008077C
:105F4000FFF807FFF8040808040808040808040814
:105F500008043E0804000806001801006000000064
:105F600004000807FFF807FFF80408080408000405
:105F70000800040800043E0006000006000001803E
:105F800000000000000000003F8001FFE00380707F
:105F90000600180400080402080402080203F007BF
:105FA00083F000020000020004000807FFF807FF6A
:105FB000F8040808000800000800000800000800B5
:105FC00004080807FFF807FFF804000800000000B5
:105FD000000004000804000804000807FFF807FF99
:105FE000F804000804000804000800000000000095
:105FF000000000000006000007000001040001048A
:10600000000104000307FFFE07FFFC04000004007A
:106010000004000004000807FFF807FFF8040C085C
:10602000001800003E0004C7800503C80600F804FD
:10603000003804001800000804000807FFF807FFF4
:10604000F80400080000080000080000080000082C
:1060500000000800001800006000000004000807AD
:10606000FFF807800807FC00007FC00003F8000766
:10607000C000780007800807FFF807FFF804000851
:1060800004000807FFF807000803C00000E0000054
:106090003800001E000007000001C00400F007FFE8
:1060A000F8040000000000007F8001FFE003807022
:1060B0000600180400080400080600180300300158
:1060C000FFE0007F8000000004000807FFF807FFE2
:1060D000F804040804040004040004040004040098
:1060E000060C0003F80001F00000000000000000B2
:1060F0007F8001FFE00380700600880400880400B0
:10610000C806003C03003E01FFE6007F840000005B
:1061100004000807FFF807FFF80408080408000453
:106120000C00040F00040BC00610F003F03801E06F
:106130000800000800000001E0F803F0300630100D
:10614000041808041808040C08040C0802061802B5
:1061500007F00781E0000000018000060000040055
:106160000004000004000807FFF807FFF804000817
:106170000400000400000600000180000400000785
:10618000FFE007FFF004001800000800000800000E
:106190000800000800000804001007FFE0040000E9
:1061A00004000006000007E00007FE00041FE000F6
:1061B00001F80000380001E0043E0007C0000600BE
:1061C0000004000004000007E00007FFC0041FF8FF
:1061D0000007C007F80007FF80043FF80007C0046D
:1061E000F80007000004000000000004000806009A
:1061F0001807C07805F1C8003E00001F800463E85E
:106200000780F806001804000800000004000006DB
:10621000000007800007E008047C08001FF8000762
:10622000F800180804E00807000006000004000059
:106230000000000100080600380400F80403E80428
:106240000F08047C0805F00807C0080700180400C0
:1062500060000000000000000000000000000000DE
:106260000000003FFFFE200002200002200002206C
:1062700000022000020000000000000000000800F2
:106280000007000000C0000038000006000001C048
:1062900000003000000E00000100000000000000BF
:1062A0000000200002200002200002200002200046
:1062B000023FFFFE000000000000000000000000A0
:1062C0000000000000000000000800001000003086
:1062D0000000200000300000100000080000000056
:1062E00000000000000001000001000001000001AA
:1062F0000000010000010000010000010000010099
:10630000000100000100000100000000000000008A
:10631000002000002000001000001000000000001D
:10632000000000000000000000000000000000006D
:1063300000F00019F8001B180022080026080024AD
:1063400008002410003FF8001FF8000008000018A3
:1063500000000004000007FFF80FFFF0001818000D
:106360001008002008002008003018001FF0000F5F
:10637000C00000000000000007C0001FF00018303F
:10638000002008002008002008003C08001C100025
:1063900000600000000000000000000007C0001FB7
:1063A000F000381800200800200800200804101011
:1063B00007FFF80FFFF000001000000000000000D1
:1063C00000000007C0001FF0001230002218002259
:1063D00008002208003208001E10000E20000000F5
:1063E00000000000200000200800200801FFF80342
:1063F000FFF80620080420080420080720000300F6
:106400000000000000000000000E000E6E001FF3F0
:106410000031B10020B10020B1003191001F130004
:106420002E1E00200E00300000000004000807FFB0
:10643000F80FFFF8001008002000002000002008DE
:10644000003FF8001FF800000800000000000000F6
:106450000000002008002008002008063FF8063F42
:10646000F80000080000080000080000000000001C
:1064700000000000000000000300000300200100F5
:106480002001002003063FFE063FFC000000000044
:106490000000000000000004000807FFF80FFFF8EC
:1064A000000188000300002FC00038F800203800E9
:1064B00020080000080000000000000000000400A8
:1064C0000804000804000807FFF80FFFF8000008A0
:1064D0000000080000080000000000000020080084
:1064E0003FF8003FF8001008002000003FF8003F90
:1064F000F8001008002000003FF8003FF8000008F6
:10650000000000002008003FF8003FF800100800DD
:106510001000002000002008003FF8001FF80000D5
:10652000080000000000000007C0000FF000183055
:106530000030080020080020080030080018300053
:106540000FF00007C0000000000000002001003F25
:10655000FF003FFF00101100200900200800200864
:10656000003038001FF0000FC000000000000000E5
:1065700007C0001FF0003818002008002008002085
:1065800009001011001FFF003FFF00000100000084
:10659000002008002008002008003FF8003FF80015
:1065A000080800100800200800200000300000301B
:1065B00000000000000000000000000C78001E1821
:1065C00000330800230800210800218800219800DA
:1065D00030F00038600000000000000020000020C3
:1065E0000000200000FFF003FFF800200800200852
:1065F0000020080000300000000000000000000043
:106600002000003FF0007FF80000180000080000A4
:1066100008002010003FF8007FF00000100000008C
:10662000000000002000003000003C00003F80001F
:1066300023F0000078000070002380003C00003050
:1066400000002000002000003C00003FE00023F894
:106650000000E0002700003E00003FE00021F800BD
:1066600001E0003E000020000000000020080020A3
:1066700008003838003E680027800003C8002CF866
:10668000003838002018002008000000000000003A
:106690002000003003003C01003F830023EC000099
:1066A00070002380003C000020000020000000005B
:1066B0000000000000000038080020380020F8002A
:1066C00023E8002F88003E0800380800201800004A
:1066D000700000000000000000000000000000004A
:1066E0000000000008000014001FF7FC3000062026
:1066F0000002000000000000000000000000000098
:1067000000000000000000000000FFFFFF0000008C
:106710000000000000000000000000000000000079
:1067200000002000023000061FF7FC0014000008E3
:106730000000000000000000000000000000000059
:106740000000001800006000004000004000002031
:1067500000001000000800000400000400000C000D
:1067600000100000B5E70200020002007FF04210B6
:1067700042107FF0421042107FF0420002080208EF
:1067800001F800000000D7D37FF000200040008017
:1067900001000200FFF802000200020002000200F5
:1067A00002000E0000000000BCBC102010201020D1
:1067B00013FEFC201020102015FC18843088D048CF
:1067C00010501020105051882606CAF501000120F3
:1067D000011001107FFC03800540054009201110C5
:1067E000210841040102010001000100D2BA008029
:1067F000404027F8114001408278424816A81AD03C
:106800002350222042204250028800000000BEA7F0
:106810003FE020203FE020203FE00000FDF8850819
:106820008508FDF885088508FDF88508000000004A
:10683000B2E200084F8828880AA88AA84AA80AA8AD
:106840002AA82AA842284508848888881038000089
:106850000000CAD44050204820400FF80040E040DB
:1068600027402240224022202A2833A82E18000840
:1068700000000000B3CC00001BF0E210221023F057
:10688000F800200033F068806080A3F02080208032
:1068900027F800000000D0F2020001003FF82000BD
:1068A0002FF02020224021803FF820882090408037
:1068B0004080838000000000D1D5200010F87E20A9
:1068C000444028F87E8848A850A864A848A872A820
:1068D00084501888610800000000C9AB1000100047
:1068E0003FE0404080807FF04210421042107FF035
:1068F0004000400840083FF800000000CCEE208037
:106900002FF8208027F0F41027F0241027F024100F
:1069100027F03410CFF80220041000000000B3E488
:1069200004000200FFF80800104020207FF00890CB
:1069300008800880088010882088C0780000000047
:10694000CEC4040002000200FFF81040104008808E
:10695000088005000200050008803060C0180000B3
:106960000000D7D604000200FFF8800880083FC06E
:10697000008001000200FFF80200020002000E0089
:1069800000000000CFD43FE0202020203FE0202066
:1069900020203FE008804890289028A008800880A8
:1069A000FFF800000000CABE00003FE00000000049
:1069B0000000FFF802001240122022104208820854
:1069C00002000E0000000000CDBC7FF84008440823
:1069D00047C84848548843084CC8733840884C0816
:1069E000430840887FF800000000C6AC008020808B
:1069F000208020803FF02000200020003FC0204069
:106A0000204020404040804000000000B4A52040CD
:106A10003840484091F07D50555055507D5055F0CC
:106A200054407C40545057F88C0800000000C3FECE
:106A30002220222027F8FA2027F0241027F03410F3
:106A4000E7F020802FF821402220EC180000000001
:106A5000CAE440804140F22044108BE8A000F7884F
:106A600024A827A834A8E7A824A8248825B80000CB
:106A70000000C8EB0800040004000200020005004A
:106A80000500088008801040104020204010800839
:106A900000000000C8AB02000200050008801040A2
:106AA0002020DFD8020002001FC002000200020006
:106AB000FFF800000000B3CC00001BF0E210221031
:106AC00023F0F800200033F068806080A3F020807D
:106AD000208027F800000000BCBC2080208020809F
:106AE000F7F02080208027E03220E2202140208023
:106AF00021402220EC1800000000CAF502000240EC
:106B000002200200FFF807000A800A8012402220BB
:106B1000421082080200020000000000D6A7020016
:106B20000200FFF8020002007FE010201040088001
:106B300005000200050018C0E03800000000B3D6D0
:106B40002080208023F0F880208027F82820302023
:106B5000E7F82020222021202020E0E00000000093
:106B6000D7A8020002007FF004000400FFF808002C
:106B700010003FE0002000401C8003000080000067
:106B80000000D7A201004080200017F00080808024
:106B90004080008017F010802080208040804FF8D7
:106BA00000000000C5FA204024402440F44824504E
:106BB000276024403440E4402440244025482648AF
:106BC000E43800000000B7A2020022202210440096
:106BD0007FF8040008000FE0142024404280810068
:106BE00006C0383800000000B3C900A00090008043
:106BF0007FF8408040907C90449044A044A044485A
:106C000058A84118820800000000B9A60100010040
:106C1000F90023F02110211021102110211039102A
:106C2000C21002100410086000000000D2C600006C
:106C3000002000780CE47904516810307E601998C7
:106C40001A3C2FE448E40838003000600000D1A16D
:106C500000000120012003FC62203420042003FCFA
:106C6000240021B021202220323E18000FE0000035
:106C7000D4F10000000010FC1304110C3DF8703E2C
:106C800010D015907CF0503E18101BFE02300020F2
:106C90000000CFEE0000000003FE00607C4012FC0C
:106CA00011041106113611241F44794400C0009CC0
:106CB00001860000C4BF000000000FE03C1820085F
:106CC00020043E04600460047E046004200C20085C
:106CD0001FF001800000B6CC0000080011FC103E3F
:106CE0003EF82D8C2904490409043E8C50FC108880
:106CF0001EC811FC100E0000B0B40000004000607F
:106D000012FE13023A427F4410C41BFE3C9871905D
:106D1000113011A00078004C0000C8B700000040FE
:106D200000F878C41F8C313821EC2126413A7DE2ED
:106D3000272225FA3D26012401040000B6A8000000
:106D4000010001705FFC700420042FF801001100A5
:106D5000113821C431003F0063E040380000B3A483
:106D6000000000000818086008C00B001E00181C76
:106D70007FF01000118010E01838098E0F0000001D
:106D8000B0B400000040006012FE13023A427F449B
:106D900010C41BFE3C987190113011A00078004C7B
:106DA0000000B7B50000000007F80600240014F842
:106DB000078C04042408261825F0647C64C2208013
:106DC0001FC00000BBD8000000001FF030182008D2
:106DD000278C2C44284428442CC427842004300CBD
:106DE0001FF803800000C7B60100210821083FF802
:106DF00000202220223EFF42229422103E10221028
:106E000022283E2822440082CABD00480044004493
:106E10000040FFFE004000403E400840084008207F
:106E200008220F12780A20060002BFAA00007FFC89
:106E300008200820082008200820FFFE082008203D
:106E4000082008201020102020204020B7A2010098
:106E50001110110822003FFC0200040007F80A0884
:106E60000908111010A0204040A003181C06CDF8FE
:106E700000007FFC40044004421452944A544424CD
:106E800044244A544A545294610440044014400833
:106E9000D6D001000100010001003FF821082108BF
:106EA0002108210821083FF8210801000100010004
:106EB0000100CEC4020001000100FFFE10101010FE
:106EC00008200820044002800100028004400820BD
:106ED0003018C006B2E2000427C414441454855488
:106EE00045544554155415542554E5542104228421
:106EF000224424140808CAD4002820241024102076
:106F000007FE0020F02017E01120111011101510BD
:106F100019CA170A02060002000000000000000063
:106F20000000000000000000000000000000000061
:106F300000000000000000000000B4F300000000AA
:106F400000000018000010000010000010000010E9
:106F50000000100C3FFFFE00100000180000180099
:106F600000340000340000220000620000410000F4
:106F7000C1800080C001006006003808001C30009D
:106F800000000000D4BD0000000000000300C002AB
:106F900000B00200980260881F888C020FF0020C7B
:106FA00080022C887FDC88030C901B0CD01B0C60AB
:106FB00013EE60131E64130CF413019C1B020C27C8
:106FC000040421D800407FFC4007F8000000B4B45E
:106FD00000000000000003800803000C02E00C0623
:106FE000300C04198C08088C08008C18208C2FF0A9
:106FF0008C48208C08208C08208C08208C08608C01
:1070000009C10C08080C08080C08080C0C0C0C072B
:10701000FC78000010000000D0C20000000000005A
:1070200002000801003C0133C03EC20008620004B7
:107030004200048200049A0C3FFFFE01023001026C
:10704000300112301FE2300102300D42301936306B
:107050001114302114302108304710300220300044
:107060000000D2BA00000000000000060018030073
:107070000C020C04FDF001198001110042330832AA
:1070800022F812421812651004E490056AB0056AED
:10709000200A71200861403860C01860C018616023
:1070A00018623018641E087800000000BEA70000B7
:1070B0000000000001004001FFC00100400100404D
:1070C00001FFC001004001004001FFC0010040007D
:1070D00000001064081FE7F8104608104608104624
:1070E000081FC7F81046081046081046081FC7F8C2
:1070F000104608000000C6C10000000000000800A3
:10710000000FFFF80C00180C00180FFFF80C40904F
:107110000C30C00C10800C11100DFFF808308008E6
:10712000308008308808309C1FFFE010208010203D
:10713000802060802040804080800300800000002C
:10714000B2E200000000000011000C09FE080D86EC
:107150000805864801A64841B64833B64813B648E4
:1071600015B64805B64805B64805B64809A6480903
:10717000A64839A448182048185808184408188602
:1071800008190238060018000000CAD400000000E8
:1071900000000001A01001D80800880C008804003D
:1071A0008400FFFE0000800000800400803C02801C
:1071B000047DC00408C0040840040840044860047A
:1071C0008822050F3407381406E01C04000E000066
:1071D00006000000000000000000000000000000A9
:1071E000000000000000000000000000000000009F
:1071F000000000000000000000000000000000008F
:10720000000000000000000000000000000000007E
:10721000000000000000000000000000000000006E
:1072200030313233343536373839204142434445E2
:10723000464748494A4B4C4D4E4F50515253545576
:10724000565758595A206162636465666768696A6F
:107250006B6C6D6E6F707172737475767778797A06
:1072600000000000847200080000002424000000D8
:10727000624E0008A872000824000024E40B0000FD
:10728000724E00080090D0030090D0030000000070
:1072900000000000010000001000000000000000DD
:0872A0000000FFFF1F00FFFFCB
:040000050800029954
:00000001FF
